:100000000C94FB0D0C94230E0C94230E0C94511B9A
:100010000C94230E0C94C41A0C94230E0C94230EEF
:100020000C94230E0C94230E0C94230E0C94A01706
:100030000C94230E0C94230E0C94230E0C94230E7C
:100040000C94FA150C94230E0C94230E0C94230E8E
:100050000C94230E0C946D1B0C94230E0C94230E05
:100060000C94411A0C94230E9224B224F3240B25F1
:100070003325332533259125912591259125390E59
:10008000400E4E0E610E6F0E7D0E8B0E88108E1080
:10009000CC102C11BC10CF104211EF10DE10E61066
:1000A000EF10DE10EF10DE108112CA12C212201300
:1000B00020132013C6121A140000190032004B003E
:1000C00065007E009700B000C900E200FC00150149
:1000D0002E01470161017A019301AD01C601E001E2
:1000E000F90113022C024602600279029302AD026A
:1000F000C702E102FB0215032F03490363037D03DB
:100100009803B203CD03E70302041D04380453042B
:100110006E048904A404BF04DB04F60412052D0553
:100120004905650581059D05BA05D605F3050F0648
:100130002C06490666068306A106BE06DC06FA06FC
:1001400018073607540773079107B007CF07EE0764
:100150000E082D084D086D088D08AE08CE08EF0872
:1001600010093209530975099709B909DC09FF0912
:10017000220A450A690A8D0AB10AD50AFA0A1F0B32
:10018000450B6A0B910BB70BDE0B050C2C0C540CBA
:100190007D0CA50CCE0CF80C220D4C0D760DA20D8D
:1001A000CD0DF90D260E530E800EAE0EDD0E0C0F8A
:1001B0003C0F6C0F9D0FCE0F0010331066109A107D
:1001C000CE10031139117011A711DF11181252123C
:1001D0008C12C812041341137F13BE13FE133F1475
:1001E0008114C31407154D159315DA1523166D16D2
:1001F000B81604175217A117F21744189818ED18DB
:1002000044199D19F719541AB21A121B741BD81BE2
:100210003E1CA71C121D7F1DEF1D611ED71E4F1F08
:10022000C91F4720C8204D21D4216022EF228123FD
:100230001824B4245325F825A1264F270228BB28CB
:100240007A29402A0B2BDE2BB82C992D822E742F65
:100250006F30733181329A33BF34EF352C377738B2
:10026000D1393A3BB43C413EE03F95415F43434581
:1002700040475B49944BEF4D70501953F055F75878
:10028000365CB15F71637C67DD6B9F70CE757C7B84
:10029000FF7FFF7FFF7FFF7FFF7FFF7FFF7FFF7F6E
:1002A000FF7FFF7FFF7FFF7FFF7FFF7FFF7FFF7F5E
:1002B000FF7FFF7FFF7FFF7FFF7F04104080C0E054
:1002C000F0FC000005000E001B002E004D007B001E
:1002D000C3003201DD01E4027904E806A80A6F10C8
:1002E00054190001FF02FF00FE0101FE00FF02FFA2
:1002F0000100040507023084808080808080808037
:1003000080808080808080808080808080808080ED
:1003100080808080808080808080808080808080DD
:1003200080808080808080808080808080808080CD
:1003300080808080808080807F7F7F7F7F7F7F7FC5
:100340007F7F7F7F7F7F7F7F7F7F7F7F7F7F7F7FBD
:100350007F7F7F7F7F7F7F7F7F7F7F7F7F7F7F7FAD
:100360007F7F7F7F7F7F7F7F7F7F7F7F7F7F7F7F9D
:100370007F7F7F7F7F7F7F7F32535658595A5B5CE8
:100380005D5D5D5E5E5E5E5E5E5E5E5D5D5D5D5D95
:100390005C5C5B5B5B5A5A5B04F4F2F0EEEDECEBF9
:1003A000EAEAE9E9E8E8E8E8E8E8E8E8E8F24A4EF5
:1003B000505253545556575812F9F8F6F5F4F3F3D2
:1003C000F2F2F2F1F1F1F1F1F1F0F0F1F1F0F1F11D
:1003D000F0F1F1F1F0F1F1EF93888685838282826A
:1003E0008181818081818181818282828293EAED13
:1003F000EFF2F3F4F5F6F6F663686B6D6F727476F0
:10040000797A3500010507F28C9295999CA0A4A7F2
:10041000ABAEB2B5B8BCBFE049494C4E515356598A
:100420005B5D606265676B53ECF2F4F7F981808481
:10043000888B8F93979B9DB528272B2E3133363988
:100440003B3E404346494C3FCED4D7DADEE1E4E7B9
:10045000EAEDF0F4F7FAFD000205080B0E11141690
:10046000191C202225282B26B0B4B7BBBEC1C4C896
:10047000CBCFD2D5D9DCDFE6307F7F7F7F7F7E7E1A
:100480007E7E7D7D7D7D7C7C7C7C7B7B7B7A7A7AAD
:100490007A7979797978787B0BD2D3D3D3D3D3D3C4
:1004A000D3D4D4D4D4D4D4D4D4D4D4D5D5D5D5D508
:1004B000D5D5D5D5D5D5D6D6D6D6D6D6D6D6D6D6E2
:1004C000D6D7D7D7D7D7D7D7D7D7D7D7D7D8D8D8BA
:1004D000D8D8D8D8D8D8D8D8D8D9D9D9D9D9D9D995
:1004E000D9D9D9D9D9DADADADADADADADADADADA71
:1004F000DADBDBDBDBDBDBDC80828486888A8C8EEC
:1005000090929496989A9C9EA0A2A4A6A8AAACAEFB
:10051000B0B2B4B6B8BABCBEC0C2C4C6C8CACCCEEB
:10052000D0D2D4D6D8DADCDEE0E2E4E6E8EAECEEDB
:10053000F0F2F4F6F8FAFCFE00020406080A0C0ECB
:1005400010121416181A1C1E20222426282A2C2EBB
:1005500030323436383A3C3E40424446484A4C4EAB
:1005600050525456585A5C5E60626466686A6C6E9B
:1005700070727476787A7C7E0306080B0D0F121564
:10058000181A1D1F222427292C2F313436383B3EC0
:1005900040434547494C4E51535557595B5E606245
:1005A000646667696B6D6F71727444C780A4D3E928
:1005B000E8E2E3EF000B0C0600FAECBCA3ADBDC60D
:1005C000C8C9CCD4DCE0E1DFDCDAD9D9D9DADBCBBD
:1005D000A594A1B4BBBCBABCC1C7CBCCCBCACACB57
:1005E000CCCED0D2D4D7D9DCDFE2E4E6E8E9ECEE39
:1005F000F0F2F4F7F9FCFE008D81818385888B8E03
:1006000092969B9FA3A8ADB2B7BCC1C6CBD0D5DA9A
:10061000DFE4EAEFF4F9FE02070C11161B20252A8D
:100620002F3417E1E3E7EAEEF2F7FBFF03080C11C2
:10063000161B1F24292E3333E4E2E5E9EDF0F4F92B
:10064000FD01050A0F13181D22262B3035F8E1E4B1
:10065000E7EAEEF2F7FBFF03080C11161B1F252A31
:100660002E33383D41464B5055595E63686C71419D
:100670001D1F2226292D3134353C4145494D50530B
:1006800055585B5D5F626466686A6C6E7071737505
:1006900077787A7C7E7F7F5A060404040406070874
:1006A0000A0B0D0F11131517191B1D1F21242629C5
:1006B0002B2D2F3234363826CBCACACBCCCDCED058
:1006C000D2D4D6D8DADDDFE1E4E6E9EBEEF0F3F5FB
:1006D000F8FAFDFF010405F88A8786868788898AEB
:1006E0008C8E90929496989A9D9FA2A4A7A9ABAE47
:1006F000B0B3B6B8BBBEC0C4FBF4EEE8E2DCD9D6FA
:10070000D3D0C5BCB7B3C1C9CACAAB9B9895C1D831
:10071000DBDEA6888887D1F9FD00A487898CF81CC8
:100720001F22BA989CA10D353636D8B7BDC41837EC
:100730003531F6E2E9EF121C16100A04FFFB162A07
:10074000303500E4E2E12B565A5D02DDDEE046740E
:10075000767714EBEFF2537F7F7D1B03060B6077F8
:1007600074702B191B1D4F5B56502B1F1F1E2F31F2
:100770002A2416100C07050000060C13191F252B40
:1007800031363C41474C51555A5E62666A6D707312
:1007900075787A7B7D7E7E7F7F7F7E7E7D7B7A789B
:1007A0007573706D6A66625E5A55514C47413C36AE
:1007B000312B251F19130C0600FAF4EDE7E1DBD508
:1007C000CFCAC4BFB9B4AFABA6A29E9A9693908D80
:1007D0008B888685838282818181828283858688D7
:1007E0008B8D9093969A9EA2A6ABAFB4B9BFC4CAA4
:1007F000CFD5DBE1E7EDF4FA010D1A262E31312FCA
:100800002D2B2B2D343C4757626C727473706B65C3
:10081000616063686F777E7F7F7F7F7F786D645EC6
:100820005C5C6064686C6D6A63594D40342A2320B7
:100830002022242626231B0FFEEDE1D7D3D3D4D6C6
:10084000D9DAD7D1C9BEB2A598928F9092979DA1BF
:10085000A2A09C92898281818181818890989FA2A7
:10086000A29F9A9592909297A0ADBBC7D1D8DBDC9E
:10087000DBD8D6D6D9DFE9F70F2B312D2B2E31302F
:100880002F3234343335373837393C3D3D3E4244DE
:1008900044464C505054657B7F705B4F4C49423D01
:1008A0003C3B373332312E2B2A2A28252424221F81
:1008B0001E1F1E1A181C1C0CF0D7CFD3D5D1CFD0B9
:1008C000D1CFCCCCCDCBC8C8C9C7C4C3C3C1BEBCB3
:1008D000BCBAB4B0AFAA9B878090A8B2B4B7BDC26F
:1008E000C4C5CACDCECFD1D4D6D6D8DBDCDCDDE1D1
:1008F000E2E1E2E7E8E5E3F1BC80FE030303030382
:1009000003030303030303030303030303030303B7
:1009100002020202020202020202020202020202B7
:1009200002020202020202020202020201010101AB
:1009300001010101010101010101010101010101A7
:100940000101010101010101010101010101010197
:100950000101010101010000000000000000000091
:100960000000000000000000000000000000000087
:100970000000000000000105F9DDC9C2C8D9F20A73
:100980002954737F78603C10E6BEA3959298A8C561
:10099000E90A28404F5551443018FEE5D4C8C2C377
:1009A000CBD9EAFC0D1B272D2D281F1405F8EDE5EA
:1009B000E0DFE1E8F0F9010A11161816130D060040
:1009C000F9F4F1EFEFF2F5FAFF03070A0C0C0B084C
:1009D0000501FFFCF9F8F7F8F9FBFE000204050633
:1009E0000605030200FFFDFCFBFCFCFDFE0000020F
:1009F00002030303020100000C1A20211F1D1A1B11
:100A00001B191613100D0C0E10100E0C0B09080AF2
:100A10000B0B0A09080707090B0B0A080605040750
:100A20000909070503020103060605030201000484
:100A3000070706030100FF000303020000FFFF0099
:100A40000304020100FFFE0002020100FFFEFEFFA0
:100A500000000000FFFEFE0003030200FFFEFE0098
:100A600003030100FFFDFDFF010100FFFEFEFACBC5
:100A700097808495ACC6DEF6000000000000000000
:100A80000000000000000000000000000000000066
:100A90000000000000000000000000000000000056
:100AA0000000000000000000000000000000000046
:100AB0000000000000000000000000000000000036
:100AC0000000000000000000000000000000000026
:100AD0000000000000000000000000000000000016
:100AE0000000000000000000000000000000000006
:100AF0000000000000000000CEB09D8283B7D80047
:100B00001EF101160E0818F2D8D7F9E3CACCD8BFE7
:100B1000CAEFE7E1FBF60411ECF1FADFD8C0A598C3
:100B2000B3B6E21D1DF7EAE2CEF10DF90B17E0C0F6
:100B3000B9CCD7EF0F1A260D1F420E19F7EFFC485C
:100B40005328223A5D54310E0AE6E9F8FE3D634728
:100B500059797F7722011E3921FDEF190C051BF70A
:100B6000BE0A1DF3CCD7F6D0EC343D1E0B22323E2C
:100B7000564713FDD9FA2C1450525F6E6D3BF7F7B0
:100B8000F7F7C48082838486C4DF1A56551CFDFDA6
:100B9000FDFD324C4B4B4A4948481FFDFDA7A6A717
:100BA000A8A8E93C3B3B3A3A00E2F80E0E0E0E0EC6
:100BB0000E0EF02022222122CECAE1FF0357555506
:100BC00054534C4242414013CBCCCCCDCD022524D2
:100BD000242429E2E2E3E3E3E4E4B28485B4FCFC08
:100BE000FCFCCE8F909192BD080808080808080800
:100BF0000807F0FBFBFBFCFA03090F161C22272D4C
:100C000033381AE7D4D655585C6064676A6C6F71E4
:100C10007375767778FC878E9090917B7F7D7B785B
:100C200075726E6B67635E5A554BEBFC02070B0FD8
:100C3000101214120F0B0702FCF6F0EAE4DFDBD708
:100C4000D3D3D3D6D8DBE0E5EBF6C4989592908D5C
:100C50008C8A8988878787878727777474766C83DF
:100C6000898C9093979BA0A4A9AFB4B9BEC4094D39
:100C70003921DDE4EBF1F7FD517B7F1E03CCD1265A
:100C8000F2FB005123670A140A6063C68BE402CCAE
:100C9000B69FF8300E4DE8E16F243FDE043BDD03E4
:100CA00035D1D96706FEFFA85375580CFEAF6320F7
:100CB0005F0D747EEF677F65A1809510858CF19E36
:100CC000DD954D06F8AC8AA3540604FC962332CE7B
:100CD000FC27C6FA26C4DC8E1B1CB8F2D0035F4D7D
:100CE00037FF157547A19DF2EBF99BDEAFFD0512AD
:100CF000D92D3801E9838486202E0F02F3D5D8EE52
:100D0000F308262B00DCCFC6C8ED36432A18EA9438
:100D100088A2BEE41735352A2C3937383818FAE658
:100D2000CBC0E300184157371A07F6F31D3F483C84
:100D300020EFD3C8CF243F525624F1BD80A0D1F577
:100D40002052463617F5DAF7E8DF1BF3E6F2C9C59D
:100D5000041D28596C2E04F0C0AAF801F04C39C5C6
:100D6000DAFAB1C1352D023208BAD5DCA9E732135F
:100D7000074016BEBFE5CFDD08253B52697A7F7F6D
:100D80007F7F7F7F7F7B6E5D4D3D2E21140A03FEAA
:100D9000FBFAFAFBFE0105080B0D0C0B080300FA29
:100DA000F3EDE4DCD7CFC9C4BFBDBEBEC0C3C6CA65
:100DB000D1D6DCE2E8F0F6FD060C131A20262B3122
:100DC000373B3D414242433F3B362F272219100B10
:100DD00004FFFBF5F3F2F2F3F7FAFE010405040356
:100DE00000FBF3E9DCCFC0B0A090848081818180DA
:100DF00080818B9DB5CCE3FDAD88858091A6989BC5
:100E0000B4BCB9BEB0968E92949FA4938388949CF0
:100E10009F9B8E92A9C3DBFA0C13130F06FAF0EA1C
:100E2000E9EDF7030C1012151A1C1B1A16100B080B
:100E30000605060605050301FFFDFDFCFCFCFCFBA9
:100E4000F8F4EFEAE7E6E7EAEFF1F3FB0711181928
:100E5000150C02F7F0EEF2FF17344E67756D636301
:100E600066727F745F5B676A6F6D5642423F42599C
:100E70006758617577727322111E20212222232464
:100E80002425252525252525252424242323222220
:100E9000212120201F1E1D2B46453E38322D28249F
:100EA000211E1C1A18161514131211100F0F0E0EF6
:100EB0000D0D0C0C0B0A0A152B2D27221D191411D0
:100EC0000F0D0B09080706050404030302020101C4
:100ED00001010000010304DC91808184888C9196DB
:100EE0009A9EA3A7ACB0B4B7BBBFC3C7CACDD1D479
:100EF000D7DADEE1E4E6E9F8D48C808B969A9FA8F5
:100F0000ABA7A29EA1AAB6C4D0D9DCDBD8D8DFEDAE
:100F1000F90410151613100E0D0A050409141D22EC
:100F2000262929251C100701FCF8F8F7F4ECE7E85E
:100F3000F1F9FBFB031C2612EADBE8FF05050811AB
:100F40001919130B09090704FEF8EFE3DBD7D8DB07
:100F5000DFE5EEF9FDFBF6F4F3F1EDEBEDF2FF0A60
:100F600015232929262428323D4B5760615D5754AB
:100F7000575F6468747E6D300A1D2D3C4B59646D5B
:100F80007578756D5D4A3B312C2E343D4852585C66
:100F90005B5854514C443A2F241B16141313141449
:100FA000120D03F6E0C7B3A3989393959799979280
:100FB0008B8380848E9EAFC1D5E9FA0A1B2B3945FD
:100FC00050585A564D413833343A41474942321805
:100FD000F6D3B8A69E9FA6AFBCC8D4DFEBF7000837
:100FE0000F110E06F7E3D2C6BEBBBCC0C5C8C8C54C
:100FF000BEB8B5B9C3D3E3F519405A6C787D7F7E8E
:101000007C7B7B7B7B7A7771675A4A362009EED3EB
:10101000BDAB9C9088838284888E959EA8B3BFCAFE
:10102000D5DFEAF5FF0A16212B353F49545E676E7E
:1010300074787A7A766E6355443019FFE3CCB7A59D
:10104000978D868382838485868686888C94A3B9CF
:10105000D6F9224963747D7F7F7D7C7D7A6F552729
:10106000EBA5859FE6376F7644FBC29D8A84848614
:101070008787888E9BB0CEF1DB9A809ED918342169
:10108000E6A38599D7183829F0AC8A9AD51138305B
:1010900001BD909AD20F3A3609C69596C80D3B3BD2
:1010A00012CF9B97C60A39421ADFA598C307384565
:1010B00022E7AB99B9FC374A2FF4BCAAC500374BDD
:1010C0003705D8C2D607374B3C14EDD8E60832496D
:1010D000422300EDF5103245422B0E00021831413B
:1010E00040301C101220303B3C3428202128303660
:1010F00037332F2E2F31301109313B2527392EFC64
:10110000D0C8D9DDC6CCF005091D393C322802B360
:101110008590A0A2B9E2FBF0D6D1F81D2A2F363572
:10112000241002F7F9131A00FA1A2C1E141813FDD2
:10113000E3DAE4F401121616284C6F75727D700D17
:1011400098808B898DB1D7E7EAEDFB0B1C251B0539
:10115000EFE8EDE2D2E50902E9F0070900F4DECCA0
:10116000CBD3D6E3072B2A12041D465C607079515D
:101170000CDBCEC4C8E1F5F923E5FFCF832931EAC2
:101180003E300B35B8EE61CFB8F4C9FE06E56B42D0
:10119000DF14FB0631ADD22FB3B02A234317E74348
:1011A00014CD0DFCE00190D25302FA4C1920F6CF79
:1011B0003716ADD9DAE51DDC237A00D7290313F9F8
:1011C000BEF1FAAEE21F3A4AF1F158FCBE2901D550
:1011D000E19CE353FE1B3D0E2BE1C0670995F5CB67
:1011E000D820DE357FEBF015EE3AEEA620E5900331
:1011F0001C325DDB0351DBDD2F6A7F7D74717477F8
:10120000757372736A470BC594828184868B949D33
:101210009F98909CC50341677577736857443D4517
:1012200059685C2FF5BFA19AA0B0C5D9E5DEC6A864
:1012300096A8D609324545381E04F5F810365B6A83
:101240005327FFE4E0ED031D2E3120FACAA297AF29
:10125000D1EBF2E7D3BFB1AFB9D7104F74755B4193
:10126000353B506572766E5620D99F848BA0ABA813
:10127000998A83828591AFE705111C27333D485336
:101280005E60ECFA0510B1A3B0BBC8D4E0EBF70286
:101290000D18242F3A4450EEE1EDF9030E1A2616EC
:1012A000B6C3D0DBE6F3FF0915202B350AC8D4DF1F
:1012B000EBF7010C18242E3944F8D6E2EFFA0410AB
:1012C0001C20ACB9C6D1DCE9F5000B17222C384341
:1012D0004D575CE8F4FF0AAD9DAAB7C3CEDBE7F239
:1012E000FD08141F2935404B56616B7418808D9989
:1012F000A6B3BFCAD7E3EEF968417741864195416D
:10130000A541B441C341D241E141F14100420F4204
:101310001E422E423D424C425C426B427A428A421D
:101320009942A842B842C742D742E642F642054334
:10133000154324433443434353436243724381433D
:101340009143A143B043C043D043DF43EF43FF4346
:101350000E441E442E443E444D445D446D447D4441
:101360008D449C44AC44BC44CC44DC44EC44FC443C
:101370000C451C452C453C454C455C456C457C4525
:101380008C459C45AC45BC45CC45DC45ED45FD4513
:101390000D461D462D463D464E465E466E467F46F0
:1013A0008F469F46AF46C046D046E146F1460147CC
:1013B000124722473347434754476447744785479A
:1013C0009647A647B747C747D847E847F9470A4867
:1013D0001A482B483C484C485D486E487F488F4827
:1013E000A048B148C248D248E348F44805491649E4
:1013F0002749384949495A496B497C498D499E4991
:10140000AF49C049D149E249F349044A154A264A3D
:10141000374A484A5A4A6B4A7C4A8D4A9E4AB04AE1
:10142000C14AD24AE34AF54A064B174B294B3A4B7D
:101430004C4B5D4B6E4B804B914BA34BB44BC64B0F
:10144000D74BE94BFA4B0C4C1D4C2F4C414C524C9A
:10145000644C764C874C994CAB4CBC4CCE4CE04C1D
:10146000F24C034D154D274D394D4B4D5D4D6E4D95
:10147000804D924DA44DB64DC84DDA4DEC4DFE4D0C
:10148000104E224E344E464E584E6B4E7D4E8F4E71
:10149000A14EB34EC54ED84EEA4EFC4E0E4F214FD4
:1014A000334F454F574F6A4F7C4F8F4FA14FB34F2C
:1014B000C64FD84FEB4FFD4F10502250355047507C
:1014C0005A506C507F509150A450B750C950DC50C6
:1014D000EF500151145127513A514C515F51725103
:1014E00085519851AB51BD51D051E351F65109523C
:1014F0001C522F524252555268527B528E52A15268
:10150000B452C852DB52EE520153145327533B538B
:101510004E536153745388539B53AE53C253D553A8
:10152000E853FC530F54235436544A545D547154B9
:1015300084549854AB54BF54D254E654FA540D55C5
:101540002155355548555C55705583559755AB55C4
:10155000BF55D355E655FA550E56225636564A56BD
:101560005E56725686569A56AE56C256D656EA56AB
:10157000FE56125726573A574F57635777578B5790
:101580009F57B457C857DC57F157055819582E586C
:10159000425856586B587F589458A858BD58D1583F
:1015A000E658FA580F59235938594D596159765907
:1015B0008B599F59B459C959DE59F259075A1C5AC7
:1015C000315A465A5A5A6F5A845A995AAE5AC35A7D
:1015D000D85AED5A025B175B2C5B415B565B6B5B29
:1015E000815B965BAB5BC05BD55BEB5B005C155CCA
:1015F0002A5C405C555C6A5C805C955CAA5CC05C63
:10160000D55CEB5C005D165D2B5D415D565D6C5DF0
:10161000815D975DAD5DC25DD85DEE5D035E195E77
:101620002F5E455E5B5E705E865E9C5EB25EC85EEF
:10163000DE5EF45E0A5F205F365F4C5F625F785F5C
:101640008E5FA45FBA5FD05FE65FFC5F12602960C7
:101650003F6055606B6082609860AE60C560DB6023
:10166000F16008611E6135614B61626178618F6173
:10167000A561BC61D261E961006216622D624462BB
:101680005A62716288629F62B662CC62E362FA62F9
:10169000116328633F6356636D6384639B63B26326
:1016A000C963E063F7630E6425643C6453646B6450
:1016B00082649964B064C864DF64F6640D6525656E
:1016C0003C6554656B6582659A65B165C965E06581
:1016D000F865106627663F6656666E6686669D6686
:1016E000B566CD66E566FC6614672C6744675C6783
:1016F00074678C67A467BC67D467EC6704681C6870
:1017000034684C6864687C689468AC68C468DD6858
:10171000F5680D6925693E6956696E6987699F6933
:10172000B869D069E969016A1A6A326A4B6A636A00
:101730007C6A946AAD6AC66ADE6AF76A106B296BC6
:10174000416B5A6B736B8C6BA56BBD6BD66BEF6B80
:10175000086C216C3A6C536C6C6C856C9E6CB86C2C
:10176000D16CEA6C036D1C6D356D4F6D686D816DCC
:101770009B6DB46DCD6DE76D006E196E336E4C6E62
:10178000666E7F6E996EB26ECC6EE66EFF6E196FEE
:10179000336F4C6F666F806F9A6FB36FCD6FE76F6B
:1017A00001701B7035704F70697083709D70B770D9
:1017B000D170EB7005711F71397153716E71887141
:1017C000A271BC71D771F1710B72267240725A729C
:1017D00075728F72AA72C472DF72F97214732E73EB
:1017E000497364737E739973B473CF73E97304742C
:1017F0001F743A74557470748A74A574C074DB7461
:10180000F67411752C75487563757E759975B47588
:10181000CF75EB75067621763C76587673768E76A4
:10182000AA76C576E176FC76187733774F776A77B4
:101830008677A277BD77D977F57710782C784878B6
:10184000647880789B78B778D378EF780B792779AC
:1018500043795F797B799779B379CF79EC79087A95
:10186000247A407A5D7A797A957AB17ACE7AEA7A70
:10187000077B237B407B5C7B797B957BB27BCE7B3C
:10188000EB7B077C247C417C5E7C7A7C977CB47CFF
:10189000D17CEE7C0A7D277D447D617D7E7D9B7DB4
:1018A000B87DD57DF27D107E2D7E4A7E677E847E5A
:1018B000A17EBF7EDC7EF97E177F347F527F6F7FF3
:1018C0008C7FAA7FC77FE57F028020803E805B807F
:1018D00079809780B480D280F0800E812C814981FC
:1018E00067818581A381C181DF81FD811B8239826E
:1018F000578276829482B2820100020004000800BE
:1019000010002000400080000001000200040000E0
:10191000190032004B0065007E009700B000C9003E
:10192000E200FB0014012D0146015F0178019101E5
:10193000AA01C301DC01F5010E022702400259028F
:1019400072028B02A302BC02D502EE0206031F0341
:1019500038035003690381039A03B203CB03E30303
:10196000FC0314042C0444045D0475048D04A504D4
:10197000BD04D504ED0405051D0534054C056405BD
:101980007C059305AB05C205DA05F10508061F06BF
:1019900037064E0665067C069306AA06C106D706DC
:1019A000EE0605071B07320748075E0775078B071A
:1019B000A107B707CD07E307F9070E0824083A087F
:1019C0004F0865087A088F08A508BA08CF08E40808
:1019D000F8080D09220937094B095F0974098809BC
:1019E0009C09B009C409D809EC09FF09130A260AA1
:1019F0003A0A4D0A600A730A860A990AAC0ABF0AB3
:101A0000D10AE40AF60A080B1B0B2D0B3E0B500BF8
:101A1000620B740B850B970BA80BB90BCA0BDB0B76
:101A2000EC0BFC0B0D0C1E0C2E0C3E0C4E0C5E0C2D
:101A30006E0C7E0C8E0C9D0CAC0CBC0CCB0CDA0C22
:101A4000E90CF80C060D150D230D320D400D4E0D51
:101A50005C0D690D770D850D920D9F0DAC0DB90DC7
:101A6000C60DD30DDF0DEC0DF80D040E100E1C0E7F
:101A7000280E340E3F0E4B0E560E610E6C0E770E76
:101A8000810E8C0E960EA10EAB0EB50EBF0EC80EBB
:101A9000D20EDB0EE40EEE0EF70EFF0E080F110F46
:101AA000190F210F290F310F390F410F480F500F18
:101AB000570F5E0F650F6C0F720F790F7F0F850F39
:101AC0008B0F910F970F9C0FA20FA70FAC0FB10FA9
:101AD000B60FBB0FBF0FC40FC80FCC0FD00FD40F62
:101AE000D70FDB0FDE0FE10FE40FE70FEA0FEC0F6C
:101AF000EF0FF10FF30FF50FF70FF80FFA0FFB0FC2
:101B0000FC0FFD0FFE0FFF0FFF0F00100010001065
:101B100000000000000000000000000000000102C2
:101B2000030405060708090A0B0C0002040507094F
:101B30000B0C00000000000002030507080B0C005E
:101B4000000000000002030507080A0C0000000066
:101B50000000020406080A0C000000000000000259
:101B600003050608090B0C00000000000204070929
:101B70000C0000000000000000030506070A0C002E
:101B800000000000000002030506090A0C00000026
:101B900000000004070C000000000000000000002E
:101BA00003070C000000000000000000000306090D
:101BB0000C00000000000000000004080C00000001
:101BC00000000000000000070C0000000000000002
:101BD000000000000C0000000000000000000000F9
:101BE000000C0707070608050607030304030201A4
:101BF0000FF0322C312C11241FBECFEFD8E0DEBF06
:101C0000CDBF24E0A8E5B1E001C01D92A33AB20720
:101C1000E1F711E0A0E0B1E0E4EEF9E602C00590E2
:101C20000D92A835B107D9F71DE0CAEFDDE004C079
:101C30002197FE010E945E31C93FD107C9F70E947A
:101C40005D1E0C94E5340C940000CF93DF93442385
:101C500009F473C0DC015B96EC914E2F50E04730E5
:101C6000510508F06AC0EC01FA01E15CFF4F0C94E9
:101C70005E3181E080936101DF91CF910C94381A3D
:101C8000EE81FF8160E0848195810E949C188F5FC6
:101C9000482F4F70EE81FF8160E00DC0EE81FF8123
:101CA00061E0848195810E949C188F5F482F43706A
:101CB000EE81FF8161E084819581DF91CF910C9469
:101CC000B418EE81FF8163E0848195810E949C18A5
:101CD0008F5F482F4F70EE81FF8163E0ECCFEE8184
:101CE000FF8165E0848195810E949C188F5F482F59
:101CF0004F70EE81FF8165E0DECFEE81FF8166E00F
:101D0000848195810E949C188F5F482F4F70EE81CF
:101D1000FF8166E0D0CFEE81FF8167E0848195810D
:101D20000E949C188F5F682F6F70EE81FF81848105
:101D30009581DF91CF910C94E218DF91CF910895B6
:101D4000BF92CF92DF92EF92FF920F931F93CF93A8
:101D5000DF938C01EA01643099F4DC011696ED9171
:101D6000FC9117972FE0249FC001259F900D11240F
:101D700064E0969587956A95E1F7978F868FFFC007
:101D8000611115C0DC011696ED91FC9117972FE0BB
:101D9000249FC001259F900D112454E096958795AE
:101DA0005A95E1F795A384A381E084ABE8C067303E
:101DB00009F0BBC0FC01838D99EF980F963008F0B5
:101DC0005EC0E80FF11DD384D8011696ED91FC9109
:101DD000179784819581FC01F4806D2D0E949C18D9
:101DE000B82ED8015B969C91993069F040F49730F9
:101DF00051F09830B9F4ED2EE694E69429C09D3068
:101E000088F4ED2E25C0CC24C394C115B8E0DB07BF
:101E100008F4C12CCC0FCD2FCC1FDD0BD195EC2FAE
:101E2000EF70EE2E2F2D30E00D2C02C0359527954A
:101E30000A94E2F72170C21659F0D8011696ED9176
:101E4000FC9117974C2D6D2D848195810E94681807
:101E5000EB1409F494C0D8011696ED91FC911797F4
:101E60004E2D6D2D84819581DF91CF911F910F9122
:101E7000FF90EF90DF90CF90BF900C94B4188D300E
:101E800079F5D8010680F781E02D440F551FC40F66
:101E9000D51FCD2FC695C69583A5C81709F46FC069
:101EA000C3A759968C915997882309F468C0149652
:101EB0008D919C9115976C2F0D960E947B16D801E1
:101EC0001496ED91FC911597E852FF4F81E090E058
:101ED00002C0880F991FCA95E2F7918380834FC093
:101EE0008E3091F424E0D695C7952A95E1F70480C9
:101EF000F581E02DE85BFF4F80858C1709F43FC02A
:101F000081E08187C0873BC08F30C9F594E0D695CA
:101F1000C7959A95E1F70480F581E02D80A58C178F
:101F200071F181E081A7C0A72AC084E0569547954A
:101F30008A95E1F7F801E60FF11D6285D801169642
:101F4000ED91FC9117970480F581E02DDF01A60F3C
:101F5000B11D15964C9382859385009781F0DC0125
:101F6000ED91FC910480F581E02DDF91CF911F91DF
:101F70000F91FF90EF90DF90CF90BF900994DF9189
:101F8000CF911F910F91FF90EF90DF90CF90BF9076
:101F90000895FC01623091F028F4662341F061302D
:101FA00041F00895633089F06430B1F0089540A3A2
:101FB000089550E05595479541AF089580E2489FB8
:101FC000A001112450A747A304C0A785B0891C967F
:101FD0004C9381E084AB089550E05595479542AF0E
:101FE0000895EF92FF920F931F93CF93DF93EC012D
:101FF000F62EE42E83E0681761F1861738F0662329
:1020000011F1A2E06A1351C04BA34FC0B4E06B17AB
:1020100009F441C085E0681348C0EF85F889468718
:1020200017A610AA11AA12AA13AA14AA15AA16AAC8
:1020300017AA10AE11AE12AE13AE14AE15AE16AE98
:1020400081E08CAB32C04F83CE0106960E94AF195F
:102050002CC04BAF8C819D818E010F5E1F4F44239E
:1020600061F021E02AA763E00E949C18E82FF0E0CD
:10207000EE0FFF1FEE53FD4F06C063E00E949C1859
:102080008AA7E2ECF2E085919491998F888FC8013C
:102090000E94FF160AC08B859C85DC01ED91FC91A6
:1020A0000084F185E02D642F09958A85F81211C00E
:1020B0008B859C85DC01ED91FC910280F381E02D04
:1020C0004E2D6F2DDF91CF911F910F91FF90EF90CB
:1020D0000994DF91CF911F910F91FF90EF90089598
:1020E0008F929F92AF92BF92EF92FF920F931F93A6
:1020F000CF93DF93EC01062F142F862F90E08730CB
:10210000910508F0D2C0FC01EA5BFF4F0C945E31F0
:102110004E83CE0106960E94AF19C7C0137084E0AB
:10212000810F21E030E0B90102C0660F771F8A9568
:10213000E2F78BA9861709F4B8C06BAB60935D0119
:1021400080915D01815080930401EFA5F8A960831F
:102150008FEF860F8183E12CFF24F394C7010E9447
:102160004A3164836BA9E9A9FAA9638370E0C701C6
:102170000E944A31628399C017708B859C85E12F3C
:10218000F0E0E654FD4F6491DC01ED91FC91048098
:10219000F581E02D099589C019A24AA386C0EF8474
:1021A000F888F7014587842F90E0FC013597E730E8
:1021B000F105E8F4E35BFF4F0C945E31812C33EFC3
:1021C000932E33EBA32E30E4B32E11C02EE5822ED6
:1021D0002FE2922E2EEFA22E20E4B22E08C099EA12
:1021E000892E9EE9992E93EEA92E9FE3B92E20E029
:1021F00030E040E855E4C501B4010E94D2310E94AC
:102200007331D7011F966D937D938D939C93529755
:10221000C501B4010E94453220E030E040E855E4B9
:102220000E94D2310E947331F701638B748B858BCE
:10223000968B17A610AA11AA12AA13AA14AA15AA55
:1022400016AA17AA10AE11AE12AE13AE14AE15AE8A
:1022500016AE81E08CAB29C0EC81FD81848183FFC7
:102260000FC0E42FF0E0EE0FFF1FEE53FD4F8591FE
:102270009491998F888FCE0141960E94FF1615C0C8
:102280004AA713C04EA7411103C01CA681E00CC091
:10229000842F83708C5F8CA781E0942F9695969500
:1022A00001C0880F9A95EAF78DA78A85081315C093
:1022B0008B859C85DC01ED91FC910190F081E02DF6
:1022C000412F602FDF91CF911F910F91FF90EF90E1
:1022D000BF90AF909F908F900994DF91CF911F9105
:1022E0000F91FF90EF90BF90AF909F908F900895C7
:1022F000CF93DF93FC01623011F160F46623B9F1F2
:10230000613009F066C00480F581E02DE15EFE4F8A
:1023100083E01BC06330D9F0643009F05AC0A48157
:10232000B581A15EBE4F82E08C9380910A0490E05B
:10233000880F991F20E030E060E070E045C0048025
:10234000F581E02DE15EFE4F81E0808342C0A481F3
:10235000B581A15EBE4F81E08C930680F781E02DB0
:102360000480F581E02D948194FF33C010C0A481D6
:10237000B581A15EBE4F82E08C930680F781E02D8F
:102380000480F581E02D848184FF23C081E0809367
:102390006101DF91CF910C94381AA72FBB27A65F5C
:1023A000BC4FAC91C681D7810884D985C02D4981A5
:1023B0005A814115510521F0EA01C20FD31FA883AC
:1023C000680F791F2F5F3F4F2038310531F710928A
:1023D0006101DF91CF910895EF920F93CF93DF9337
:1023E000611121C0FC01218D21111DC0EC018481EE
:1023F0009581865E9E4FFC0120814985213021F424
:10240000EE24E39402E003C022E0E22E01E0242F58
:1024100068E00E94EF1DEC81FD81E357FF4F808152
:10242000813009F48A8FDF91CF910F91EF90089559
:10243000DC011696ED91FC91179762858481958158
:10244000FC01448150E0062E02C0559547950A9440
:10245000E2F741705527F1E04F2741700C9468185E
:10246000CF92DF92EF92FF920F931F93CF93DF9360
:10247000CDB7DEB7C158D1090FB6F894DEBF0FBE95
:10248000CDBF8C01DC011696ED91FC911797F2847B
:1024900014960D90BC91A02DFD01E957FF4F0190BE
:1024A000F081E02D611123C2A65EBE4F413019F4C8
:1024B00082E08C9346C291E0E13DF74008F490E061
:1024C00012961C921297E0EFFBE1E49111968C9129
:1024D0001197E823EC93F801A481B5816D01F6EE24
:1024E000CF1AFEEFDF0A81E0F60180834F2D50E026
:1024F0004830510508F025C2FA01EC5AFF4F0C9400
:102500005E31D8015A968C915A97882309F43EC0BF
:102510005A961C925A971696CD90DC901797B6E073
:10252000CB0ED11C00E010E0E12CF12C80919E0438
:102530008111FCCF80919D048111F8CFDE011196AD
:1025400080E090E0B701600F711FFC01E60FF71FFC
:10255000E850FD4FE491ED93019680389105A9F77D
:10256000CE0101960E94341EE0E8EE0EF11CE1144B
:10257000F8E0FF06D9F6185F011520E11207A1F671
:10258000C6013EC0F801828D81113DC0C8010E9484
:102590001812D7C1D8011696ED91FC91179799237F
:1025A00059F18781668170E0B0E18B9F600D711DEC
:1025B00011247695762F662777956795CE0101963B
:1025C0007C0140E050E000851185D80111960D9105
:1025D0001C9112970115110521F0040F151FD80148
:1025E0002C91D7012D937D014F5F5F4F40385105EE
:1025F00051F70E94341EA5C110926101CF010696C9
:102600000E9481199EC1128E1D968C911D9781305A
:1026100071F02CF4811195C168EF73E00AC082302B
:1026200061F0833009F08DC16EEF73E002C06AEF94
:1026300073E0CD010E943C1D84C16CEF73E0F9CFC3
:10264000F801818D882309F467C01D969C911D9720
:10265000F4E0FF1679F025E0F216E1F0D8011696C5
:10266000ED91FC91179793A7998341E050E067EFB4
:1026700073E018C0F801938F973020F481E05F96E3
:102680008C9302C05F961C92998341E050E066EF04
:1026900073E008C0AB5DBE4F9C93998341E050E06E
:1026A00065EF73E0CE0101960E946034D80159961F
:1026B0001C925997ED91FC911197C484D58416967C
:1026C000ED91FC9117976F2D848195810E949C1844
:1026D000482F6F2DC801F6010995D8018D919C9165
:1026E000119716960D90BC91A02D14960D90BC914B
:1026F000A02D14964C9150E00F2C02C05595479593
:102700000A94E2F74170DC011E96ED91FC911F974F
:102710006F2DC801099515C1992309F437CF81E0C0
:10272000F801818F93E0F60190831D968C911D979F
:10273000F4E0FF1689F125E0F21609F453C09CE09D
:1027400053969C9353978C301CF08BE01D968C9382
:10275000D8011696ED91FC91179714968D919C9146
:10276000159763A50D960E947B16D8011496ED91DE
:10277000FC9115979F0128523F4F16960D90BC91E2
:10278000A02D81E090E09B960C9002C0880F991FCD
:102790000A94E2F7F90123C090E153969C93539772
:1027A00080311CF08FE01D968C93D80114968D918A
:1027B0009C9115975B966C910D960E947B16D801A3
:1027C0001496ED91FC911597E852FF4F81E090E04F
:1027D0005B960C9002C0880F991F0A94E2F79183D0
:1027E0008083AFC024E053962C935397843014F029
:1027F0001D969C93F80184819581FC01EB5DFE4F51
:1028000060810D960E947B16D80114968D919C9143
:102810001597DC01A852BF4FFC01EB5DFE4F81E034
:1028200090E0008002C0880F991F0A94E2F78D9310
:102830009C9387C0D8011696ED91FC91179767E09D
:10284000992399F1848195810E949C18D80116964C
:10285000ED91FC9117970480F581E02DBAE08B9FF4
:10286000B00111248081898381818A8382818B8355
:1028700083818C837F0125E0E20EF11C9E012B5F9A
:102880003F4FCF010A96D7014D917D01D9014D935C
:102890009D01E816F906B9F784818A874AE050E07D
:1028A000CE0101960E9460340EC0848195810E9401
:1028B0009C18D8011696ED91FC911797682F84818A
:1028C00095810E94E218D8011696ED91FC91179718
:1028D00067E0848195810E949C18898341E050E0E3
:1028E00064EF73E0CE0101960E9460342AC061302B
:1028F00041F5413031F5AC57BF4F8C91811121C06A
:10290000F801818D81111DC040936101CF57DF4FC8
:102910004883C158D0400E94381AD8011496ED91CE
:10292000FC911597E957FF4F80819181CF57DF4F79
:102930004881C158D040813D974018F0D8015A963F
:102940004C93CF57DF4F0FB6F894DEBF0FBECDBF0D
:10295000DF91CF911F910F91FF90EF90DF90CF907B
:1029600008950F931F93CF93DF93EC016A87EB8554
:10297000FC850190F081E02D008111818C819D8189
:102980000E949C18482F6A858B859C85F8010995C3
:102990008B859C856A85DC01ED91FC91AC81BD81C4
:1029A00014964C9150E0062E02C0559547950A9416
:1029B000E2F741700280F381E02DDF91CF911F910A
:1029C0000F910994FC01611110C0218D86819781BE
:1029D000211103C0642F0C94B11424813581FC01B2
:1029E0006285C90102960C947B166130C9F4818D11
:1029F000811108C00680F781E02D62858481958170
:102A00000C94B4180480F581E02DE852FF4F81E06A
:102A100090E002C0880F991F4A95E2F79183808366
:102A200008954F925F926F927F928F929F92AF9292
:102A3000BF92DF92EF92FF920F931F93CF93DF939A
:102A4000EC01162F2BAD4E96222309F450C00E94A4
:102A50005318BC01CE018A960E94881629893A89AA
:102A60008217930779F02D893E898217930751F0D9
:102A70009A8B898B3C8B2B8B1D8E1C8ECE014196A5
:102A80000E94FF168D899E8929893A8982179307AA
:102A900021F1EA8DFB8D3097E9F0AC8DBD8DA10F52
:102AA000B11DBD8FAC8FEA17FB07A0F00B891C8905
:102AB000A90160E070E09A01AB01201B310B4109D4
:102AC00051090E94A1349F0140E050E00E948234ED
:102AD000200F311F3E8B2D8B07C02B893C89281777
:102AE000390711F09C8B8B8B8D899E890DC02AA58F
:102AF000222341F00E945318BC01CE018A960E9405
:102B0000881602C00E9453189EAB8DAB8DA99EA95A
:102B10000E94261898AF8FABABA9B0E0B595A795EA
:102B2000B595A7959C010E946C314B015C010D8508
:102B30001E85F80180819181A281B3818816990652
:102B4000AA06BB0609F444C080829182A282B382A5
:102B5000E12CF12C412C84E2582E84EF682E712C4C
:102B6000C301B2010E2C04C0660F771F881F991F86
:102B70000A94D2F7A50194010E94B434C9012F3FF1
:102B8000310551F048F021E030E001C0220FEA9415
:102B9000EAF72093020107C0FFEFEF1AFF0A28E0CF
:102BA000E216F104E9F60197909301018093000188
:102BB00081E080930D0420910201F801948129178E
:102BC00028F490910201948380935C0181E08CABA6
:102BD000DF91CF911F910F91FF90EF90DF90BF9009
:102BE000AF909F908F907F906F905F904F900895DF
:102BF0000E94EF331F920F920FB60F9211242F9362
:102C00003F938F939F93AF93BF938091580190917F
:102C10005901A0915A01B0915B013091180423E051
:102C2000230F2D3720F40196A11DB11D05C026E804
:102C3000230F0296A11DB11D209318048093580103
:102C400090935901A0935A01B0935B0180911404B1
:102C500090911504A0911604B09117040196A11D3E
:102C6000B11D8093140490931504A0931604B0939F
:102C70001704BF91AF919F918F913F912F910F902A
:102C80000FBE0F901F9018951F93CF93DF93EC0109
:102C9000DB0120E08C91281750F56981822F0E947A
:102CA0002A3111964D915C911297911117C04115DF
:102CB000510521F0FA01E20FF11D30818881E32FE7
:102CC000032E000CFF0B082E02C0F595E7950A9421
:102CD000E2F71E2F01C0110F8A95EAF74115510541
:102CE00021F0420F511DFA0110832F5FD3CFDF91E6
:102CF000CF911F910895FC01868168171CF08150C7
:102D00008083089567FF02C010820895608308954C
:102D10000F931F93CF93DF93FC01EB01218140ECD4
:102D20004203900111243D5FC901860F971F60E0A7
:102D300073E00E943631DC01208130E0F901E0527D
:102D4000F44E94918DE0829F8001839F100D112499
:102D5000F801E05FF44EE49180E4E89FB0011124B3
:102D600080E098170CF440C0292F092E000C330B7B
:102D7000281B310987FD339537FF02C02F5F3F4F76
:102D800035952795280FF801E20FF11D27FDFA95DB
:102D9000E05FF44E449130E4439FA00111244A17B0
:102DA0005B0738F481E0820F9D01241B350BA901DC
:102DB00007C0A417B507C8F49FEF920F4A1B5B0B1F
:102DC000A617B70720F49B012A1B3B0B03C09D01EC
:102DD000261B370B4217530708F0C3CF649130E42A
:102DE000639FB0011124BDCFAB01CE018A1B9B0BA9
:102DF000840F951FDF91CF911F910F910895CF936D
:102E0000DF93EC01AF81B885109719F41A86198603
:102E100022C08E818823E9F0488159818A819B8173
:102E2000EC81FD818417950738F49A012E1B3F0B26
:102E30000E94D6349F0106C09F01241B350B0E94BF
:102E4000D6349A0140E050E00E94B4343A87298792
:102E500002C0BA87A987DF91CF910895CF93DF93FE
:102E6000FC018185882319F0118681E001C080E092
:102E700023813481458156814217530720F4D901BB
:102E8000A41BB50B03C0DA01A21BB30B97819923D6
:102E900011F19081519738F0911105C091E0908324
:102EA000128211820EC0992361F0A181B281ED01DD
:102EB000C60FD11DBE01D283C183603D774008F0AB
:102EC00010829081992379F02417350761F03683B9
:102ED000258381E008C0AB2B29F081E08083368315
:102EE000258301C01082DF91CF910895FC01FF2757
:102EF0008F3F910559F050F0811522E0920768F458
:102F000080E091E09C012E1B3F0BF901EE0FFF1FAB
:102F1000E25FF64E8591949108958115934030F0CB
:102F200080E091E09C012E1B3F0BF901EE0FFF1F8B
:102F3000E25FF64E8591949191958195910908955E
:102F40001F920F920FB60F9211242F933F934F931E
:102F50006F937F938F939F93AF93BF93EF93FF9361
:102F600080910D04882349F060910201809113043F
:102F70000E942A31992309F45AC030911304311167
:102F80000FC080915C01882331F081E08093600163
:102F900010925C0105C08091600181111092600166
:102FA00080916001E0910B04F0910C048823D1F032
:102FB000A0915E01B0915F0111968D919C91129745
:102FC000009721F0DC01A30FB11D2C91818192812A
:102FD000009721F0FC01E30FF11D2083205820937E
:102FE000B4000BC081819281009721F0FC01E30FB6
:102FF000F11D408140584093B4009091040120910C
:10300000050180911304820F892380931304FF919B
:10301000EF91BF91AF919F918F917F916F914F9160
:103020003F912F910F900FBE0F901F901895809198
:103030000001909101019093890080938800809114
:1030400002018093050110920D0497CFCF93DF9377
:103050009C01C0E0D3E0BE010E943631FB01EE0FBF
:10306000FF1FE850F74EA591B4916C9FC0016D9F72
:10307000900D7C9F900D1124F901E81BF90BEE0FC8
:10308000FF1FE850FD4E259134910E94D634DC019B
:10309000CB0129E0B695A795979587952A95D1F705
:1030A000DF91CF910895FC0183819481208131814A
:1030B000280F391F8281280F311D85818111305FD2
:1030C000C901813C2FE1920710F080EC9FE1089547
:1030D0000F931F93FC015481442379F081E090E029
:1030E000A0E0B0E0062E04C0880F991FAA1FBB1FE6
:1030F0000A94D2F7852B84830FC001E010E020E012
:1031000030E0062E04C0000F111F221F331F0A9447
:10311000D2F700950523048382859385009749F0B3
:10312000DC01ED91FC910280F381E02D1F910F9164
:1031300009941F910F910895DC01262F2170E22F31
:10314000F0E0E051F44E849170E075956795A60F1C
:10315000B71F9C91892390E0220F220F02C0959502
:1031600087952A95E2F70895CF93DF93EC01A62F78
:10317000B0E0B595A795962F9170E92FF0E0E0515A
:10318000F44EE491AC0FBD1F2E2F20958C9182231D
:10319000990F990F242F01C0220F9A95EAF7E22385
:1031A000E82BEC938A859B85009749F0DC01ED9133
:1031B000FC910190F081E02DDF91CF910994DF9196
:1031C000CF9108956F927F928F929F92AF92BF920C
:1031D000CF92DF92EF92FF920F931F93CF93DF93E3
:1031E000CDB7DEB72A970FB6F894DEBF0FBECDBFBE
:1031F0008C018AE0689FB00111244AE050E0CE01C2
:1032000001960E945034DE0111965D01912C20EF51
:10321000C22E2BE1D22E31EFE32E3BE1F32E35010E
:10322000F6014491892C880CD5018D915D014823CC
:10323000682DC8010E94B418F7014491D3018C9104
:10324000482350E094E0559547959A95E1F761E061
:10325000680DC8010E94B4189394B4E09B12DFCFAC
:103260006801E5E0CE0ED11C84E0E82EF12C6CEF75
:103270006E0DE1E0F0E0EC0FFD1FEE0DFF1D408153
:10328000D6014D936D01F80182859385009739F041
:10329000DC01ED91FC910480F581E02D0995BFEFF3
:1032A000EB1AFB0AE9E0EE16F10409F7E12CF12C28
:1032B0004A8550E00E2C02C0559547950A94E2F7D6
:1032C00041706E2DC8010E946818FFEFEF1AFF0AC7
:1032D00087E0E816F10461F72A960FB6F894DEBF8E
:1032E0000FBECDBFDF91CF911F910F91FF90EF9057
:1032F000DF90CF90BF90AF909F908F907F906F9016
:103300000895CF93DF93DC0120E030E011968C919B
:103310001197EC91F0E090E1899FE00DF11D1124EF
:10332000F695FE2FEE27F795E795E20FF31FE8508D
:10333000FD4FE4911296CD91DC91139749815A810A
:103340004115510521F0EA01C20FD31FE8832F5F19
:103350003F4F20383105D1F6DF91CF910895CF93BB
:10336000DF93CDB7DEB7C058D1090FB6F894DEBFF2
:103370000FBECDBFDC0111964C9111972C9130916D
:103380009E043111FCCF30919D043111F8CF309162
:10339000BC0034FDF4CF30E0B0E14B9F200D311D77
:1033A00011243695322F22273795279530931B0409
:1033B00020931C0422E020931A0421E020939E0411
:1033C0001092190420911904206A2093190425EE03
:1033D0002093BC0020919E042111FCCF2091BC00C1
:1033E00024FDF8CF20E820931A0421E020939D04C7
:1033F0002093190420911904206A2093190425EEC2
:103400002093BC0020919D042111FCCF2091BC0091
:1034100024FDF8CF20E8EBE1F4E0DE011196019005
:103420000D922A95E1F7FE01319620E030E061919E
:10343000DC0112964D915C911397DA0111964D9132
:103440005C9112974115510521F0DA01A20FB31FCB
:103450006C932F5F3F4F2038310549F7C058DF4F3D
:103460000FB6F894DEBF0FBECDBFDF91CF910895A8
:1034700010920A048FE7809309048EEC80937A00FF
:1034800008951F920F920FB60F9211248F939F935E
:10349000EF93FF938091B900887F883261F168F4DF
:1034A0008031F9F028F48823D1F18830D1F063C05D
:1034B000883109F1803299F15EC0803409F442C04C
:1034C00038F4803361F1883309F055C085E928C0AC
:1034D000803559F1883509F441C0883409F04BC072
:1034E00045C0809119048093BB0085EC8093BC009B
:1034F0001092120440C09091120480911A049817FF
:1035000070F4E0911204F0E0E55EFB4F808180935F
:10351000BB00809112048F5F8093120419C084E96C
:103520008093BC0010929E0426C0E0911204F0E04B
:103530008091BB00E55EFB4F8083809112048F5F1A
:10354000809312049091120480911A04981710F439
:1035500085EC01C085E88093BC000DC0E0911204A9
:10356000F0E08091BB00E55EFB4F808384E98093AF
:10357000BC0010929D04FF91EF919F918F910F904D
:103580000FBE0F901F9018951F920F920FB60F92BB
:103590001124CF92DF92EF92FF920F931F932F93FC
:1035A0003F934F935F936F937F938F939F93AF93CB
:1035B000BF93CF93DF93EF93FF93E9B0E094C0E123
:1035C000D4E0AEE0B4E062EF72E040E050E00E2DF7
:1035D00010E0FA01EA50FD4FF490FE208881F816C1
:1035E00009F43CC0FB01849131969491F80102C02A
:1035F000F595E7958A95E2F7E170FF27EE0FFF1F3B
:10360000EE0FFF1F680102C0D594C7949A95E2F7A8
:10361000C6018170992723E0880F991F2A95E1F749
:103620008E2B9F2B2C9130E035952795359527953E
:10363000822B932B8C93FC01EE51FD4F8491FA0168
:10364000EE0FFF1FEE59FE4F208131816901C81A2C
:10365000D10887FDD394D182C082F8822196119639
:103660006E5F7F4F4130510519F041E050E0B1CF1E
:10367000FF91EF91DF91CF91BF91AF919F918F918A
:103680007F916F915F914F913F912F911F910F917A
:10369000FF90EF90DF90CF900F900FBE0F901F9094
:1036A00018951F920F920FB60F9211248F939F932C
:1036B000EF93FF9383B18095982F9170E6E6F1E048
:1036C0009083869581708183FF91EF919F918F9177
:1036D0000F900FBE0F901F9018951F920F920FB66C
:1036E0000F9211248F939F93EF93FF938091790012
:1036F00090916101913019F0923031F154C0E09114
:103700000A04F0E08058E65FFC4F8083E0910A04F1
:10371000F0E0E65FFC4F808187FD3DC0E0910A0448
:10372000F0E0E75FFC4F808187FF35C082E0809347
:103730006101E0910A04F0E0E65FFC4F8081809334
:103740000A0310920A0427C0E0910A04F0E08058AE
:10375000E65FFC4F808380910A048F3F11F483E081
:1037600017C0E0910A04F0E0E65FFC4F808187FD1E
:1037700012C0E0910A04F0E0E75FFC4F808187FF10
:103780000AC090910A0480910301981720F084E008
:103790008093610108C080910A048F5F80930A04BE
:1037A0008EEC80937A00FF91EF919F918F910F9013
:1037B0000FBE0F901F9018952A9870E062FB882723
:1037C00080F986608EBD0DB407FEFDCF8EB586E014
:1037D000660F771F8A95E1F76EBD0DB407FEFDCF2A
:1037E0002EB51EBC0DB407FEFDCF8EB52A9A2F70E4
:1037F00090E0922B0895EF92FF920F931F93CF9337
:103800007C018C01085E1F4FC0E0D8018D918D01B5
:103810008130D9F46C2FC7010E94DC1B41E081305C
:10382000984008F440E0F801E95AFF4F80814817BA
:1038300061F04083F70180819181DC01ED91FC9181
:103840000284F385E02D6C2F0995CF5FC830E9F62F
:10385000CF911F910F91FF90EF900895CF92DF923B
:10386000EF92FF921F93CF93DF93EC01162F0E94EC
:10387000DC1B41E050E0143011F440E050E0A0E0E7
:10388000B0E0E6E0E49F9001E59F300D11242C0F9D
:103890003D1FF901E858FF4F40815181841B950B72
:1038A000A109B109BC01CD01ABE0660F771F881FEC
:1038B000991FAA95D1F734962081318140E050E0DC
:1038C0000E94823469017A0184E0D80EE11CF11C67
:1038D000812F90E0F7FE0BC02AE0289FF001299F7E
:1038E000F00D1124EC0FFD1F14A213A21EC0C11471
:1038F000A0E1DA06E104F1046CF02AE0289FF0016F
:10390000299FF00D1124EC0FFD1F2FEF3FE034A392
:1039100023A30BC06AE0689FF001699FF00D11249A
:10392000B096EC0FFD1FD482C3822AE0289F70015D
:10393000299FF00C1124C701809660E08C0F9D1F19
:103940000E942E17882369F188819981DC01ED910D
:10395000FC910480F581E02DCE0DDF1D28A54BA143
:103960005CA12F3FA9F030E02F5F3F4FBA0144E048
:10397000769567954A95E1F7269FA001279F500D00
:10398000369F500D112464E0569547956A95E1F7EE
:10399000612FDF91CF911F91FF90EF90DF90CF903B
:1039A0000994DF91CF911F91FF90EF90DF90CF901E
:1039B0000895CF92DF92EF92FF920F931F93CF93D0
:1039C000DF9300D0CDB7DEB77C011A8219826B017C
:1039D00028EFC21A23E0D20A86011695079516959C
:1039E0000795112742E050E0CE0101960E94503425
:1039F000C801880F991F880F991FC81AD90AD69431
:103A0000C794F801EE0FFF1FE00FF11FEC0DF11D41
:103A1000FC96EE0FFF1FEE0DFF1D898190E0982FA1
:103A200088272A81820F911D9183808326E0209F21
:103A3000C001219F900D1124E80EF91ED701A45852
:103A4000BF4FC70186589F4FE8E7EE0EF11CFC01FF
:103A500080819181F70120813181821B930B8D93AD
:103A60009C930F900F90DF91CF911F910F91FF903A
:103A7000EF90DF90CF9008954F925F926F927F9278
:103A80008F929F92AF92BF92CF92DF92EF92FF926E
:103A90000F931F93CF93DF9300D0CDB7DEB77C0198
:103AA0003B011A821982CB018D7F883F934019F424
:103AB00074E0472E01C0412C630188EFC81A83E0EF
:103AC000D80A860116950795169507951127C801FE
:103AD000880F991F880F991FC81AD90AD694C794BE
:103AE00068E0562E812C912C5401642DC7010E9450
:103AF000DC1B880E991EA11CB11C5A945110F5CFE5
:103B000083E0B694A794979487948A95D1F7998285
:103B10008A8242E050E0B301CE0101960E946034F7
:103B2000F801EE0FFF1FE00FF11FEC0DF11DFC96E9
:103B3000EE0FFF1FEE0DFF1D9182808226E0209F79
:103B4000C001219F900D1124E80EF91ED701A45841
:103B5000BF4FC70186589F4FE8E7EE0EF11CFC01EE
:103B600080819181F70120813181821B930B8D939C
:103B70009C930F900F90DF91CF911F910F91FF9029
:103B8000EF90DF90CF90BF90AF909F908F907F90FD
:103B90006F905F904F90089590919E049111FCCF8B
:103BA00090919D049111F8CF9091BC0094FDF4CFB9
:103BB00060931B0410921C0492E090931A0491E00D
:103BC00090939E0410921904909119048062880FBA
:103BD000892B8093190485EE8093BC000895EF92A1
:103BE0000F93CF93DF93DC0112966C931297149688
:103BF0001C92149761EF7BE1FB01C49180EF9BE184
:103C0000FC01D4915C2F509513963C91139735236A
:103C1000F0E14F9FA00111244C23432B3D2F309501
:103C200043232D23422B13964C931397FB0164914E
:103C3000FC018491262F209511969C911197922337
:103C4000F0E10F9F900111242623292B982F9095A6
:103C50002923E822E22A1196EC9211970C93DF9126
:103C6000CF910F91EF900895FC0180919E048111F6
:103C7000FCCF80919D048111F8CF8091BC0084FD20
:103C8000F4CF70931B0460931C0490E8ADE1B4E0A2
:103C900001900D929A95E1F782E880931A0481E0F1
:103CA00080939E041092190480911904806A809375
:103CB000190485EE8093BC000895CF93DF93CDB7B0
:103CC000DEB7A0970FB6F894DEBF0FBECDBF7894D5
:103CD00084B5826084BD84B5816084BD85B5826011
:103CE00085BD85B5816085BD80916E0081608093C2
:103CF0006E0010928100809181008260809381002B
:103D0000809181008160809381008091800081603A
:103D1000809380008091B10084608093B100809195
:103D2000B00081608093B00080917A0084608093BD
:103D30007A0080917A00826080937A0080917A0084
:103D4000816080937A0080917A00806880937A0005
:103D50001092C100E0916C01F0916D0111E01187AA
:103D600080916E0190916F012091B6002F7B20937E
:103D7000B6002091B6002F7D2093B6002091B000B0
:103D800021602093B0002091B00022602093B00009
:103D90002091B100277F2093B1002091B0002F7EA9
:103DA0002093B0002091B00020622093B0002091B9
:103DB000B0002F7B2093B0002091B0002F7720938C
:103DC000B0002091B10021602093B1002091B1009A
:103DD0002D7F2093B1002091B1002B7F2093B10063
:103DE000F894209180002E7F209380002091800005
:103DF0002D7F2093800020918100286020938100F6
:103E0000209181002F7E20938100209181002160EC
:103E100020938100209181002D7F209381002091AB
:103E200081002B7F209381002091000130910101BE
:103E3000309389002093880020916F0022602093A6
:103E40006F007894DC01D196ED91FC91D2972FEF21
:103E500021839F96ED91FC91D097238360E00E948F
:103E6000B11441E050E067EF73E0CE0101960E948B
:103E700050348981E0916E01F0916F0183A741E098
:103E800050E066EF73E0CE0101960E9450348981C4
:103E900080938301E0916C01F0916D01873010F403
:103EA000178F01C0178E41E050E065EF73E0CE013F
:103EB00001960E9450348981E0916C01F0916D016E
:103EC000EB5DFE4F808341E050E064EF73E0CE0194
:103ED00001960E94503469816F70E0916E01F091FB
:103EE0006F01848195810E94E21840917101809157
:103EF0006C0190916D01A2E0EA2E01E0242F64E0B4
:103F0000865E9E4F0E94EF1D4091710180916C0171
:103F100090916D01EE24E39402E0242F64E0815E31
:103F20009E4F0E94EF1D8FB7F89440915801509119
:103F3000590160915A0170915B018FBF809193018B
:103F400090919401A0919501B0919601F42EF81AE8
:103F50008F0D911DA11DB11D80939301909394012C
:103F6000A0939501B093960100916C0110916D01A1
:103F70002801B8E14B0E511C6801E0E2CE0ED11CC5
:103F8000E12C4801FBED8F1AFEEF9F0A7724739412
:103F9000580128E4A20EB11CD2018D912D0181118E
:103FA00055C08E2D8B7F6E2D21F4C8010E942E1CD2
:103FB0004DC0C8010E94DC1BF601948383836F2DE2
:103FC000C6010E942E17882309F440C0D60113961B
:103FD0004D915C911497B5E0EB1215C0F40180810E
:103FE00080FF29C0F4E056954795FA95E1F7D50191
:103FF00018968C911897841749F119967C92199705
:1040000018964C9323C0B6E0EB1215C0F4018081E2
:1040100081FF11C0E4E056954795EA95E1F7D80194
:1040200098968C919897841789F099967C92999795
:1040300098964C930BC0F80180819181DC01ED9141
:10404000FC910480F581E02D6E2D0995E394BAE092
:10405000CB0ED11CE8E0EE129FCF80916C019091C5
:104060006D010E94FB1B40906C0150906D0142015C
:10407000F4E88F0E911C82010B571F4F620129E853
:10408000C20ED11CA12CB12C6F2C712CEA2CF50185
:10409000EA59FE4F4081D4014C934130E1F4F801DC
:1040A00082819381860D971D938382832681378138
:1040B0008217930780F0D6018C9181110CC04C932C
:1040C000F20180819181DC01ED91FC910280F3810C
:1040D000E02D6A2D0995F80180819581891710F4EA
:1040E0008F0D8083D8018C91891758F1F40190814C
:1040F000F60133972081921721F1913051F421116B
:104100000DC013961C921E921297D6011C9281E04C
:1041100006C0911103C081E0213009F080E0908356
:10412000F8011082882369F0D2018D919C91DC0105
:10413000ED91FC910190F081E02DD4014C916E2D18
:104140000995B9E08B0E911C075F1F4FE9E0CE0E79
:10415000D11CAA94AB2821F0AA24A394B12C96CF09
:1041600080906C0190906D0164012CE0C20ED11C16
:1041700054013AE0A30EB11C84010E5F1F4F612C65
:10418000712CEE24E394662DF301EE0FFF1FEE5920
:10419000FE4F80819181F60130812291321738F0F3
:1041A000D80112969C938E931197D6011C92D6013A
:1041B0008C919081891710F48F0D8C93F8012181D7
:1041C000328183819481A901481B590BCA0157FD93
:1041D00003969595879595958795009709F441C025
:1041E000D80114963C932E93139797FD03C0F501C5
:1041F000E08202C0D5011C92F6013597208122236E
:1042000011F1F8019081890F8083F6013397908135
:104210003197992369F09081891724F0891BD8017F
:104220008C9311C087FF0FC0890FF80180830BC0EA
:104230009081891724F09150D8019C9304C087FF86
:1042400002C0F8011082F40180819181DC01ED91BE
:10425000FC910680F781E02DD5012C91D8014C917D
:104260000995FBE0CF0ED11C2BE0A20EB11C055F1F
:104270001F4F6A94672821F066246394712C83CFC2
:10428000E0916C01F0916D0180916101909192013A
:10429000981769F06091610160939201808191812A
:1042A000DC01ED91FC910084F185E02D09952091D0
:1042B0006C0130916D01F901EC5DFE4F80818F0D35
:1042C0008083E12C8081803120F080518083E394D1
:1042D000F9CFE1101AC0E0916C01F0916D019F01DE
:1042E0002A563F4FAEE8B1E010E0AF01465E5E4FA8
:1042F0005F0161EEA61A6EEFB60AF2E1CF2E03E07F
:10430000D02E01E085EEE82E19C1B90166527F4F2B
:10431000D901A650BF4F40E050E0AE2CB12C89012E
:1043200008521F4FFB017080772009F45DC08D910A
:104330009C9111978A0D9B1D11969C938E93F80169
:10434000C080D180FB018088E1EFFBE19490E0EF39
:10435000FBE15490F601042E02C0F695E7950A940D
:10436000E2F7E0FF20C08920912CE4E09594879447
:10437000EA95E1F788159905B8F188199909119618
:104380009C938E93212C312C21012394042E04C064
:10439000220C331C441C551C0A94D2F720943094F0
:1043A0002C203D2018C08520912C88159905E0F01F
:1043B0008819990911969C938E93212C312C2101F7
:1043C0002394042E04C0220C331C441C551C0A9454
:1043D000D2F72C283D28F80131822082FFEF7F168A
:1043E00019F07A94FB0170824F5F5F4F6F5F7F4FD0
:1043F00012964031510509F095CF8901045E1E4F98
:10440000D901A25EBE4FB901665E7E4F285D3E4F68
:10441000F8018081882309F43FC0DC90DE0CDC9237
:10442000FB01A080FD0133974081E1EFFBE1849126
:10443000842390E054E0959587955A95E1F7982E5E
:10444000E0EFFBE1B490B422FD013197C080E1EFD1
:10445000FBE144914C2150E0E4E055954795EA9505
:10446000E1F7E0EFFBE17490A81202C0D41638F433
:10447000AB1012C0C720DC1478F0A91005C0D41A04
:10448000DC92FB01B08204C0DC18DC92FB0180836B
:10449000F8018081815080830B5F1F4F15966B5F01
:1044A0007F4FA217B30709F0B3CF15CFFA01608190
:1044B000762F7D7F713009F494606250623008F489
:1044C0009860F5016081762F7D7F713009F49160ED
:1044D0006250623008F492606D917C91119786175A
:1044E000970731F111969C938E9360919E04611110
:1044F000FCCF60919D046111F8CF6091BC0064FD18
:10450000F4CFC0921B0480931C0490931D04D0929E
:104510001A0400939E041092190490911904802F9C
:10452000811B8062880F892B80931904E092BC0064
:104530002E5B3F4F1296113039F011E0F901808166
:1045400091811111C9CFB2CF6F2D80916E019091E1
:104550006F010E94111520906E0130906F01D10102
:10456000D3961C911983E12EF12CC7010E94C2320F
:104570009B838A83F10180859185892B69F4D10120
:10458000D9964C91D997D196ED91FC91D2976081B3
:104590002181611156C043C0F10186818F30D1F471
:1045A0008781811117C0E12CF12CE11640F70E94A0
:1045B0004034880F892F881F990B2A813B81211550
:1045C000310521F0F901EE0DFF1D8083FFEFEF1A99
:1045D000FF0AEBCF80E890E0B7010E944A3150E03B
:1045E00080E090E040E0811750F6D1011896ED91FF
:1045F000FC911997218132812115310521F0F901B2
:10460000E40FF11D50812A813B812115310521F0F4
:10461000F901E80FF91F5083460F0196E4CF2111ED
:1046200010C0D1011496ED91FC911597848186FFFD
:104630004EC0BE016F5F7F4FC1018C960E94441631
:1046400046C070E06F5F7F4F3FE7369FC001379FE6
:10465000900D11240281892F602F0E942A31182F7A
:10466000042E000C550B57FF03C05195419551097D
:1046700030E02F5F3F4F429FD001439FB00D529FCC
:10468000B00D1124CD01880F892F881F990B9195AA
:10469000602F0E942A314381282F30E0210F311DE5
:1046A000642F70E06217730714F0482F410F80E009
:1046B00090E0841708F0B5CF2A813B8121153105A0
:1046C00021F0F901E80FF91F10820196F2CFF101F4
:1046D00083859485DC01ED91FC910680F781E02DC6
:1046E0000995F10184A9882309F4BFC514AAC10161
:1046F00084960E945318D101D5962D913C91D6975E
:10470000820F931F9C5097FF02C080E090E0813C95
:10471000BFE19B0714F080EC9FE10E942618DC01AA
:10472000F10107851089F80193878287F10185855A
:104730009685FC014080518062807380F80122815F
:10474000338144815581C484E080F180D584DD20AB
:1047500009F45BC053014201B694A79497948794DF
:104760008C869D86AE86BF869BE0992E9D14B8F4FC
:10477000C301B201E7E09695879577956795EA952D
:10478000D1F7688779878A879B8753014201F4E0D4
:10479000B694A79497948794FA95D1F711C0992766
:1047A000872D762D652D688779878A879B875301AA
:1047B000420196E0B694A794979487949A95D1F77E
:1047C0006C857D858E859F85681979098A099B0985
:1047D0004D01A12CB12C681579058A059B0528F49B
:1047E000D8011B967C936E931A97F8018285938566
:1047F000A0E0B0E088849984AA84BB8488159905D8
:10480000AA05BB0510F493868286D8011A96ED910D
:10481000FC911B97BBE0BD1538F088248394D81415
:1048200048F410928C01A4C4AFE09A2E9D1408F0B5
:10483000DBC29EC4AC2DB0E00E94A1344B015C01F0
:104840008E0C9F1CA11CB11CCF01A0E0B0E0BC01EC
:10485000CD01EAE0660F771F881F991FEA95D1F70F
:10486000A30192010E94B43480918A0190918B013E
:104870008217930791F48091860190918701A0910E
:104880008801B091890188169906AA06BB0629F409
:1048900080918C01D81609F4E8C430938B012093E1
:1048A0008A018092860190928701A0928801B0923D
:1048B0008901D0928C01C901939593702B8F3C8F05
:1048C0004D8F5E8F0E9476177C012B8D3C8DC90128
:1048D0000E9476176C01092E000CAA0BBB0BBC01C1
:1048E000CD014CE0660F771F881F991F4A95D1F7BD
:1048F000A50194010E94823449015A01B594A794FC
:1049000097948794D8011D96BC91BC878B2F90E01B
:1049100001978B30910508F02BC48C5C9F4FFC01F4
:104920000C945E3180E090E18E199F09AC015595A1
:104930004795052E000C660B770BD80193964D9387
:104940005D936D937C939697092E000CAA0BBB0B7D
:10495000F80187A390A7A1A7B2A743A754A765A76B
:1049600076A71DC0C701905F95958795092E000C0D
:10497000AA0BBB0BF80183A394A3A5A3B6A340E0A5
:1049800050EF4E195F09052E000C660B770B47A3FD
:1049900050A761A772A783A794A7A5A7B6A7D5011B
:1049A000C401905FAF4FBF4F878B908FA18FB28FA5
:1049B000EE0CFF1C882799278E199F09092E000CE1
:1049C000AA0BBB0B838F948FA58FB68F80E090E1ED
:1049D000A0E0B0E088199909AA09BB09878F90A3C4
:1049E000A1A3B2A3C5C3C60195958795092E000C56
:1049F000AA0BBB0BF80183A394A3A5A3B6A317A28C
:104A000010A611A612A6B095A095909581959F4FDE
:104A1000AF4FBF4FC0CF20E030E140E050E0D801C1
:104A200093962D933D934D935C939697EE0CFF1CBC
:104A3000882799278E199F09092E000CAA0BBB0BFA
:104A4000F80187A390A7A1A7B2A723A734A745A7DA
:104A500056A7B501A401505F6F4F7F4F478B508F12
:104A6000618F728FAFCFD8011F964D905D906D9082
:104A70007C905297A5019401C301B2010E941A31A2
:104A8000DC01CB015CE0B595A795979587955A9584
:104A9000D1F7AC01BD01505F6F4F7F4FF80143A3C9
:104AA00054A365A376A3EE0CFF1CCC24DD24CE1802
:104AB000DF080D2C000CEE08FF08C7A2D0A6E1A667
:104AC000F2A620E030E140E050E0281B390B4A0B11
:104AD0005B0B23A734A745A756A7C501B401ECE09B
:104AE000660F771F881F991FEA95D1F7A3019201DE
:104AF0000E948234DA01C901905FAF4FBF4FF801C5
:104B0000878B908FA18FB28FC38ED48EE58EF68E59
:104B100080E090E1A0E0B0E0821B930BA40BB50B0A
:104B20005DCFD8011F964D905D906D907C9052970F
:104B30006701FF0CEE08FF08A3019201C701B6014F
:104B40000E941A31DC01CB013CE0B595A795979501
:104B500087953A95D1F79C01AD012C193D094E0975
:104B60005F092C833D834E835F83AC01BD014C0DF7
:104B70005D1D6E1D7F1D488759876A877B87D80119
:104B800053966D917D918D919C915697A5019401BD
:104B90000E941A314B015C014BE0B594A7949794A5
:104BA00087944A95D1F7FC85FA5073016201B0E110
:104BB000DB0EE11CF11CA3019201305141095109A6
:104BC000288B398B4A8B5B8BF23008F484C0B70199
:104BD000A6018C819D81AE81BF81481B590B6A0B58
:104BE0007B0B4C875D876E877F87CB01BA01680D91
:104BF000791D8A1D9B1DA30192010E941A31DC01BF
:104C0000CB013CE0B595A795979587953A95D1F757
:104C1000F80183A394A3A5A3B6A3688979898A8997
:104C20009B89288539854A855B85621B730B840BBC
:104C3000950BA30192010E941A31DC01CB016BE0BC
:104C4000B595A795979587956A95D1F787A390A76E
:104C5000A1A7B2A76C857D858E859F856819790986
:104C60008A099B090E941A31DC01CB017CE0B595D1
:104C7000A795979587957A95D1F783A794A7A5A728
:104C8000B6A72C813D814E815F81C20ED31EE41EEA
:104C9000F51ED701C601880D991DAA1DBB1D878B66
:104CA000908FA18FB28F88899989AA89BB8928851D
:104CB00039854A855B85820F931FA41FB51F880F16
:104CC000991FAA1FBB1FB095A095909581959F4FE6
:104CD000AF4FBF4F80C02C813D814E815F812C0D35
:104CE0003D1D4E1D5F1D2C873D874E875F87CA0186
:104CF000B901680D791D8A1D9B1DA30192010E94B7
:104D00001A31DC01CB013CE0B595A79597958795C5
:104D10003A95D1F7F80183A394A3A5A3B6A380E0A5
:104D200090E1A0E0B0E084199509A609B709BC019B
:104D3000CD01288539854A855B85621B730B840B01
:104D4000950BA30192010E941A31DC01CB016BE0AB
:104D5000B595A795979587956A95D1F787A390A75D
:104D6000A1A7B2A76C857D858E859F856819790975
:104D70008A099B090E941A31DC01CB017CE0B595C0
:104D8000A795979587957A95D1F783A794A7A5A717
:104D9000B6A72C813D814E815F81C21AD30AE40AF5
:104DA000F50AD701C601880D991DAA1DBB1D878B69
:104DB000908FA18FB28F88899989AA89BB8928850C
:104DC00039854A855B85821B930BA40BB50B880F35
:104DD000991FAA1FBB1F838F948FA58FB68FC818EA
:104DE000D908EA08FB08AFC0CF01A0E0B0E0BC01E1
:104DF000CD0129E0660F771F881F991F2A95D1F7EB
:104E0000A30192010E94B4348091840190918501A4
:104E10008217930729F480918C01D81609F425C2D2
:104E20003093850120938401D0928C01C901992788
:104E30003D7F2F3F310509F040F4FC01EE0FFF1FCD
:104E4000E854FF4FE590F4900DC0E0E0F1E0E81B7E
:104E5000F90BEE0FFF1FE854FF4FE590F490F1942B
:104E6000E194F108BEE0DB1609F4CEC0EFE0DE16F7
:104E700009F424C147010F2C000CAA08BB088C823E
:104E80009D82AE82BF82D80116964D905D906D9046
:104E90007C901997BDE09701DB1609F45CC0D7013F
:104EA0000E9464316B017C014CE0F594E794D79447
:104EB000C7944A95D1F7F801C3A6D4A6E5A6F6A6ED
:104EC000C3A2D4A2E5A2F6A2D701C601880F991FFA
:104ED000AA1FBB1F87A390A7A1A7B2A7A5019401F2
:104EE000C301B2010E941A31DC01CB016CE0B5951F
:104EF000A795979587956A95D1F746015701880E32
:104F0000991EAA1EBB1EF0E19F0EA11CB11CF80148
:104F1000878A908EA18EB28E46015701F0E19F1ACA
:104F2000A108B108880C991CAA1CBB1CF801838E2F
:104F3000948EA58EB68EC81AD90AEA0AFB0AF0E149
:104F4000DF0EE11CF11CD8015F96CD92DD92ED924F
:104F5000FC9292970DC1D7010E9464316B017C01D4
:104F6000ECE0F594E794D794C794EA95D1F746011D
:104F70005701B0E19B0EA11CB11C20E030E140E0E4
:104F800050E0D80193962D933D934D935C93969763
:104F9000F80123A734A745A756A720E030EE4FEF2E
:104FA0005FEF97962D933D934D935C939A972C8149
:104FB0003D814E815F81C301B2010E941A31DC0143
:104FC000CB012CE0B595A795979587952A95D1F7B4
:104FD00024013501480E591E6A1E7B1E478A508ED9
:104FE000618E728EF0E1DF1AE108F108CC0CDD1C55
:104FF000EE1CFF1CF801C38ED48EE58EF68E881A47
:10500000990AAA0ABB0AADC09701D7010E94643170
:105010009B01AC016CE055954795379527956A95AE
:10502000D1F7A3E0B0E00E94A1344B015C01F8018C
:1050300063A774A785A796A7D80193966D937D93D0
:105040008D939C9396972B013C01440C551C661C38
:10505000771C47A250A661A672A623E030E0D701D4
:105060000E946C31DC01CB01905FAF4FBF4F880DC8
:10507000991DAA1DBB1D878B908FA18FB28FF0E267
:105080005F1A61087108D8015B964D925D926D922E
:105090007C925E979701ADEFBFEF0E946431DC0117
:1050A000CB01905FAF4FBF4F880E991EAA1EBB1E4B
:1050B000F801878E90A2A1A2B2A25AC09701D7018F
:1050C0000E9464314B015C013CE0B594A794979435
:1050D00087943A95D1F720E030E340E050E0D801E2
:1050E0009B962D933D934D935C939E97F80123A33C
:1050F00034A345A356A320E030EA4FEF5FEF979625
:105100002D933D934D935C939A9723E030E0D70124
:105110000E946C31DC01CB01880D991DAA1DBB1DBD
:10512000905DAF4FBF4F878B908FA18FB28FD5010E
:10513000C401880F991FAA1FBB1F9056A109B1096E
:10514000838F948FA58FB68F9701ADEFBFEF0E942D
:105150006431860E971EA81EB91EF0E39F0EA11C97
:10516000B11CD8015F968D929D92AD92BC929297A0
:10517000F801C788D08CE18CF28C83A194A1A5A101
:10518000B6A1BC01CD01ECE0660F771F881F991F07
:10519000EA95D1F7A70196010E948234D80193962F
:1051A0002D933D934D935C93969797968D919D91FA
:1051B0000D90BC91A02DBC01CD01FCE0660F771FC6
:1051C000881F991FFA95D1F7A70196010E94823492
:1051D000F80127A330A741A752A783A594A5A5A5A9
:1051E000B6A5BC01CD01ACE0660F771F881F991FE3
:1051F000AA95D1F7A70196010E948234D8019B9607
:105200002D933D934D935C939E975B968D919D91CD
:105210000D90BC91A02DBC01CD01BCE0660F771FA5
:10522000881F991FBA95D1F7A70196010E94823471
:10523000F801238F348F458F568F878D90A1A1A1C0
:10524000B2A1BC01CD012CE0660F771F881F991F0A
:105250002A95D1F7A70196010E948234D8015F9662
:105260002D933D934D935C939297F101078510899F
:10527000D8011D968C91882309F439C18980888AC8
:105280001C8A1D821C8218869801215C3F4F3A8F30
:10529000298FFC81FC87D8011E968C918888F8158F
:1052A00008F0F6C0EA81FB81F8A3EF8F309731F068
:1052B000AC81BD81AE0FBF1F8C908C8A2C89822E51
:1052C000220F9908AA08BB08882341F062E0880CE5
:1052D000991CAA1CBB1C6A95D1F707C056E0880C24
:1052E000991CAA1CBB1C5A95D1F7D8019F964D91C9
:1052F0005D916D917C91D2974D8B5E8B6F8B788F8A
:10530000D7964D905D906D907C90DA9793966D91C5
:105310007D918D919C919697A50194010E941A31DF
:105320006B017C01F80167A170A581A592A52D896B
:105330003E894F89588D0E941A31C60ED71EE81E2D
:10534000F91E23A534A545A556A563A974A985A969
:1053500096A90E941A31C60ED71EE81EF91E638D4B
:10536000748D858D968DA30192010E941A31C61A03
:10537000D70AE80AF90A278D30A141A152A163ADED
:1053800074AD85AD96AD0E941A31C61AD70AE80AE7
:10539000F90A4CE0F594E794D794C7944A95D1F76D
:1053A000C114F0E8DF06E104F1044CF4C11420E874
:1053B000D2062FEFE206F2062CF0C60105C08FEFF1
:1053C0009FE702C080E090E86C01990FEE08FF08AB
:1053D0004D895E896F89788DD801D3964D935D9301
:1053E0006D937C93D697F80187A690AAA1AAB2AA3A
:1053F000DB964D925D926D927C92DE97C7AAD0AEFD
:10540000E1AEF2AE36E0F594E794D794C7943A95BE
:10541000D1F7F0E8CF16D104E104F1044CF420E810
:10542000C2162FEFD206E206F20624F09C2D03C02E
:105430009FE701C090E8EF8DF8A1309729F08C80AC
:105440009D80E80DF91D9083D8011E968C918823CC
:1054500051F0903819F097FD919501C09FE788842D
:1054600089160CF498878C858F718F3159F4A98D2A
:10547000BA8D8D919C91DC01ED91FC910190F081B0
:10548000E02D0995EC81FD813196FD83EC8301CF00
:10549000882369F19884692D990C770B8FE790E048
:1054A0000E944A3140E020E030E0A8882A15A0F4AC
:1054B0008A819B81009721F0FC01E20FF31F40815C
:1054C000469F502D1124009721F0FC01E20FF31F9D
:1054D00050832F5F3F4FE9CFF801FF968081918184
:1054E000DC01ED91FC910190F081E02D0995D10155
:1054F0001496ED91FC9115978185882309F4CFC00E
:10550000DA964C91DA979F96ED91FC91D097628153
:105510002381611103C0222309F4C1C070E06F5FD1
:105520007F4F3FE7369FC001379F900D11240481C4
:10553000892F602F0E942A31182F042E000C550B42
:1055400057FF03C051954195510930E02F5F3F4F00
:10555000429FD001439FB00D529FB00D1124CD0149
:10556000880F892F881F990B9195602F0E942A31EF
:105570002081482F50E0410F511D622F70E06417C9
:10558000750714F0180F01C0122F111101C011E09E
:1055900090918D01892F911708F4820F811BD12CD6
:1055A000E12CF12C70E060E02981621708F074C0F2
:1055B0002A813B812115310521F0D901A60FB11DAA
:1055C0007C91072F072E000C110B20853185D90106
:1055D00011964D915C9112974115510529F09A0150
:1055E000280F311DD901FC902F2D0F2C000C330BEF
:1055F000058002C0359527950A94E2F7200F311FE8
:105600002038310534F42038BFEF3B071CF420E884
:1056100001C02FE74115510521F0DA01A90FB11D95
:105620002C93AA80BB80A114B10429F09501260F08
:10563000311DD901EC900E2D0E2C000C110B0780A2
:1056400002C0159507950A94E2F720853185D901A6
:1056500011964D915C9112974115510521F0480F1B
:10566000511DDA01DC902D2D0D2C000C330B068022
:1056700002C0359527950A94E2F7200FA114B104D2
:1056800021F0D501A60FB11D2C9321819F5F92239C
:105690008F5F82236F5F88CF90938D011286D10137
:1056A0001496ED91FC911597848186FD07C0BE018B
:1056B0006F5F7F4FC1018C960E944416D1011D96E9
:1056C000ED91FC911E9780916001811124C030E022
:1056D00020E080915D012817C0F48A819B810097AA
:1056E00021F0DC01A20FB11D3C91A0915E01B091AF
:1056F0005F0111968D919C911297009721F0DC012A
:10570000A20FB11D3C932F5FE4CF809102018483EF
:1057100081E080935C01F10183859485DC01ED914A
:10572000FC910680F781E02D09958A819B81009785
:1057300011F00E94573380E090E0892B11F40C9413
:10574000931F0E9400000C94931F6093030108951F
:10575000609303010895FC01218D21110BC0848108
:105760009581FC01E65EFE4F442311F082E001C00A
:1057700081E08083089502970C94AB2B0F931F93C5
:10578000CF93DF93DC0159962C91599721113EC09C
:105790001496ED91FC911597613039F424E0238B38
:1057A0002585243094F023E00FC0643039F428E0DC
:1057B000238B258528304CF027E006C020E1238B81
:1057C0002585203114F02FE02587042F162FEC01BA
:1057D0008C819D81642F0D960E947B168C819D810A
:1057E000FC01EA56FF4F21E030E0A90102C0440F5E
:1057F000551F1A95E2F751834083EE5BFF4F02C0BD
:10580000220F331F0A95E2F731832083DF91CF9176
:105810001F910F91089502970C94BE2BCF93DF93A5
:10582000EC018C819D810E94FB1B64E08C819D8139
:105830000E942E1C60E08E819F81DF91CF910C949D
:10584000111502970C940E2C662329F081E08093A9
:1058500061010C94381A10926101089502970C941A
:10586000242C08952F923F924F925F926F927F92D5
:105870008F929F92AF92BF92CF92DF92EF92FF9260
:105880000F931F93CF93DF9300D000D000D0CDB7FC
:10589000DEB784E391E090936901809368018EE420
:1058A00091E090936B0180936A018091BE02811117
:1058B000D4C010929A0110929C0110929B011092F8
:1058C0009E0110929D0181E080939F0190E1909351
:1058D000A0018093A1011092A2011092A301109245
:1058E000A4011092A5011092A7011092A601109296
:1058F000A9011092A8018093AA019093AB01809313
:10590000AC011092AD011092AE011092AF0188E08F
:10591000E0EBF1E0DF011D928A95E9F7E8EBF1E0B9
:1059200080E090E031E02FEF108212821182148229
:10593000138216821582DC01A856BE4F97963C93BF
:10594000979798962C93989799961C920A963A96C0
:105950008035910549F788E0E8E0F2E0DF011D922B
:105960008A95E9F78CE0E0E1F2E0DF011D928A958B
:10597000E9F710921C0210921D0210921E02109262
:10598000200210921F021092210224E6209322028C
:1059900080ED97E0909324028093230210922502D9
:1059A00010922602109227021092290210922802C9
:1059B00010922A0220932B0290932D0280932C02A6
:1059C00010922F0210922E0280E1E0E3F2E0DF015C
:1059D000882E1D928A94E9F7E0E4F2E0DF01882E38
:1059E0001D928A94E9F790E2E0E5F2E0DF01892E6A
:1059F0001D928A94E9F71092710210927002E2E708
:105A0000F2E0DF01882E1D928A94E9F7E2E8F2E0E5
:105A1000DF011D928A95E9F7E2E9F2E0DF011D92CC
:105A20009A95E9F71092B2021092B3021092B40262
:105A30001092B5021092B6021092B7021092B802FC
:105A40001092B9021092BA021092BB021092BC02DC
:105A50001092BD0281E08093BE0288E991E09093AC
:105A60006D0180936C0180910203811182C082E2FA
:105A700091E09093C7028093C6028EE291E09093EA
:105A8000C9028093C8021092CC021092CD0283E02A
:105A900090E00E94C2327C0110E8FC01108380E893
:105AA00090E00E94C232D70112969C938E93119778
:105AB000F092CF02E092CE028CEC92E00E9481192B
:105AC0001092D00288EB91E09093D8028093D70295
:105AD0009093DA028093D9029093DC028093DB02E8
:105AE0001092DD021092DF021092DE021092E102AB
:105AF0001092E0021092E3021092E2021092E5028C
:105B00001092E4021092E6021092E8021092E7026C
:105B10001092E9021092EB021092EA021092EC024B
:105B20001092EE021092ED021092EF021092F0022B
:105B30001092F1021092F20281E08093F30210922F
:105B4000F4021093F9021092FA0220E431E130934A
:105B5000FC022093FB0220EE36E03093FE022093FD
:105B6000FD021092FF021092000310920103809335
:105B7000020306EC12E010936F0100936E018EE8B1
:105B80008093700184E08093710188E0E0E1F1E0AE
:105B9000A2E7B1E001900D928A95E1F786E0E8E195
:105BA000F1E0AAE7B1E001900D928A95E1F78CE36C
:105BB00080938001109281011092820110928301E2
:105BC0008AE691E09093D2028093D1028CE090E03B
:105BD0000E94C232FC0180E3808389E1818384E1F9
:105BE0008283138214829F012B5F3F4F85E0D9018E
:105BF0001D928A95E9F713870287F093CB02E09311
:105C0000CA0281E490E00E94C232FC0180E098E088
:105C10009183808389E391E0A0E0B0E08283938365
:105C2000A483B58380EA96E1A0E0B0E08683978301
:105C3000A087B18780E197E29387828714861586D3
:105C4000168681E090E0A0E0B0E0878B908FA18F76
:105C5000B28F88EC92E0DF01DF96009719F41D9275
:105C60001C9202C08D939C93F093D602E093D502D0
:105C700085E090E00E94C2326C0180E097E3A0E0F2
:105C8000B0E0F60180839183A283B383148200E89D
:105C900000935D0180915D0181508093040183E058
:105CA00090E00E94C2327C01DC010C9380E890E01D
:105CB0000E94C232F70192838183F0920C04E09239
:105CC0000B0483E090E00E94C2327C01DC010C9363
:105CD00080E890E00E94C232F70192838183F092C3
:105CE0005F01E0925E01D092D402C092D302109183
:105CF000F90210935D0180915D0181508093040150
:105D00008BE090E00E94C2326C01DC0112961C9282
:105D1000129713961C92139781E015968C93159702
:105D200016968C93169717968C9317971A961C9223
:105D300083E090E00E94C2327C01FC01008380E895
:105D400090E00E94C232D70112969C938E931197D5
:105D5000F601F186E086D092F602C092F502108339
:105D60008FEF810F8183612F70E080E091E00E94CE
:105D70004A31648384E090E06B830E94C232FC016C
:105D80001082118213836B8162839093F802809357
:105D9000F70280906C0190906D019E828D8288E662
:105DA00091E0D4018D939C93F8942A9A229A8CB511
:105DB00080618CBD8CB580648CBD239A259A8DB58D
:105DC00081608DBD8CB58D7F8CBD8CB581608CBDA7
:105DD0008CB58F7D8CBD8CB5877F8CBD8CB58B7F52
:105DE0008CBD68EF73E08D819E810E94D91C6AEFA3
:105DF00073E08D819E810E94D91C6CEF73E08D81D0
:105E00009E810E94D91C6EEF73E08D819E810E945D
:105E1000D91C4D805E80B8E14B0E511C0D811E8156
:105E2000005E1F4FAD80BE80E7E2AE0EB11CCD809C
:105E3000DE80F8E2CF0ED11C6D807E8029E2620EFA
:105E4000711CF12CEE24E39499249A9436E0832E6D
:105E500022242A944FE0342E5A824982D2018C9116
:105E6000811172C08F2D8B7F6F2D09F060C08D81E5
:105E70009E810E94DC1B41E050E0B4E0FB1202C0B6
:105E800040E050E0A0E0B0E0849E9001859E300D9F
:105E90001124ED81FE812E0F3F1FF901E858FF4FBD
:105EA00040815181841B950BA109B109BC01CD0131
:105EB0002BE0660F771F881F991F2A95D1F734961C
:105EC0002081318140E050E00E948234DA01C90132
:105ED0009C5FAF4FBF4FB7FF0FC0D8011C92129607
:105EE0001C921E92119714961C921E92139716964E
:105EF0001C921E92159714C08115F0E19F07A10511
:105F0000B105CCF0D8011C9212961C921E921197EA
:105F100014963C922E92139716963C922E921597B9
:105F2000F501E082D6019C92F30110821BC08D81A5
:105F30009E810E94DC1BF8011082128211829483E0
:105F400083839683858308C0F801108212821182B0
:105F50001482138216821582D501EC92F60190828A
:105F6000D3011C92BFEF4B1A5B0AE981FA81808151
:105F70009201295A3F4F813089F46F2D8D819E8186
:105F80002B833C830E94DC1B41E02B813C818130D0
:105F9000984008F440E0D9014C9302C0F901108206
:105FA000F394065F1F4FFAE0AF0EB11C2AE0C20E59
:105FB000D11C4AE0640E711C58E0F5124DCFED8102
:105FC000FE81E15BFF4F1082AD81BE8197961C92EE
:105FD00010927C0080917C00806480937C00809192
:105FE0007C00806280937C0020E030E0C12CD12CCA
:105FF0007601C39400E010E0F801E20FF31FEE50C9
:10600000FD4F84914AB14601570104C0880C991C88
:10601000AA1CBB1C8A95D2F7D501C4018095909526
:10602000A095B09550E060E070E084239523A6230E
:10603000B7238AB9E4914BB1D701C60104C0880FD8
:10604000991FAA1FBB1FEA95D2F7842B8BB9013089
:10605000110519F001E010E0CFCF2E5F3F4F243043
:10606000310541F6209828982198299856985E98ED
:10607000539A5B9883B18095982F917090936601A5
:1060800090916601ED81FE81EC57FF4F9083ED8189
:10609000FE81EB57FF4F1082ED81FE81EA57FF4FE3
:1060A0009083ED81FE81E957FF4F11821082ED81CF
:1060B000FE81E757FF4F108294E6ED81FE81E6579F
:1060C000FF4F908320ED37E0ED81FE81E557FF4FD4
:1060D0003183208386958170809367018091670169
:1060E000ED81FE81E357FF4F8083ED81FE81E25712
:1060F000FF4F1082ED81FE81E157FF4F8083ED81DC
:10610000FE81E057FF4F11821082ED81FE81EE5635
:10611000FF4F1082ED81FE81ED56FF4F9083ED81A0
:10612000FE81EC56FF4F3183208380916B008160AC
:1061300080936B0080916B00826080936B00D89A93
:106140008091680081608093680080916D00846018
:1061500080936D0080916D00806180936D008091CF
:106160006D00806280936D0080916D0080648093EB
:106170006D0080916D00806880936D00DA9A809147
:10618000680084608093680088E0AD81BE811896C5
:106190008C93189712968C91129788301CF087E098
:1061A00012968C9378948091B9008E7F8093B90079
:1061B0008091B9008D7F8093B90088E48093B80006
:1061C00085E48093BC0060E080E00E94CC1D61E02B
:1061D00080E00E94CC1D60E081E00E94CC1D61E067
:1061E00081E026960FB6F894DEBF0FBECDBFDF91DB
:1061F000CF911F910F91FF90EF90DF90CF90BF90C4
:10620000AF909F908F907F906F905F904F903F9056
:106210002F900C94CC1DDC011B968D919C911C97AA
:10622000DC01ED91FC910680F781E02D0994029745
:106230000C940B31DB018F939F930E94A134BF918B
:10624000AF91A29F800D911DA39F900DB29F900DC5
:1062500011240895991B79E004C0991F961708F03E
:10626000961B881F7A95C9F780950895AA1BBB1BBA
:1062700051E107C0AA1FBB1FA617B70710F0A61B46
:10628000B70B881F991F5A95A9F780959095BC0167
:10629000CD01089597FB072E16F4009407D077FDE3
:1062A00009D00E94363107FC05D03EF490958195C7
:1062B0009F4F0895709561957F4F0895EE0FFF1FD2
:1062C0000590F491E02D09940E94D634332312F402
:1062D0008A1B9B0B0C946E310E94D634B7FF089535
:1062E000821B930B08950E947A316894B1110C942B
:1062F000CC3108950E94B13188F09F5798F0B92FA2
:106300009927B751B0F0E1F0660F771F881F991FEA
:106310001AF0BA95C9F714C0B13091F00E94CB3190
:10632000B1E008950C94CB31672F782F8827B85FA0
:1063300039F0B93FCCF3869577956795B395D9F742
:106340003EF490958095709561957F4F8F4F9F4F4C
:10635000089557FD9058440F551F59F05F3F71F055
:106360004795880F97FB991F61F09F3F79F08795BC
:106370000895121613061406551FF2CF4695F1DF45
:1063800008C0161617061806991FF1CF86957105D5
:10639000610508940895E894BB2766277727CB0109
:1063A00097F908950E94E5310C94B1320E94A3320E
:1063B00038F00E94AA3220F0952311F00C94853217
:1063C0000C94993211240C94CC310E94A93170F3B1
:1063D000959FC1F3950F50E0551F629FF001729F8A
:1063E000BB27F00DB11D639FAA27F00DB11DAA1F99
:1063F000649F6627B00DA11D661F829F2227B00DE6
:10640000A11D621F739FB00DA11D621F839FA00D70
:10641000611D221F749F3327A00D611D231F849FC0
:10642000600D211D822F762F6A2F11249F57504017
:106430009AF0F1F088234AF0EE0FFF1FBB1F661F92
:10644000771F881F91505040A9F79E3F510580F05B
:106450000C9485320C94CC315F3FE4F3983ED4F336
:10646000869577956795B795F795E7959F5FC1F7FF
:10647000FE2B880F911D9695879597F9089519F42D
:1064800016F40C9499320C948B320E94B131B8F30B
:106490009923C9F3B6F39F57550B87FF0E949C328F
:1064A0000024A0E640EA900180585695979528F47C
:1064B000805C660F771F881F20F026173707480774
:1064C00030F4621B730B840B202931294A2BA695CB
:1064D00017940794202531254A2758F7660F771F10
:1064E000881F20F026173707480730F4620B730B1C
:1064F000840B200D311D411DA09581F7B901842F1A
:106500009158880F96958795089597F99F6780E829
:1065100070E060E008959F3F31F0915020F487953E
:1065200077956795B795880F911D9695879597F9FB
:1065300008959FEF80EC089591505040660F771FAB
:10654000881FD2F7089500240A9416161706180615
:106550000906089500240A94121613061406050667
:106560000895092E0394000C11F4882352F0BB0FF8
:1065700040F4BF2B11F460FF04C06F5F7F4F8F4F5B
:106580009F4F0895CF93DF938230910510F482E0FE
:1065900090E0E091A104F091A20420E030E0C0E09E
:1065A000D0E0309711F14081518148175907C0F070
:1065B0004817590761F482819381209719F09B83D2
:1065C0008A832BC09093A2048093A10426C0211536
:1065D000310519F04217530718F49A01BE01DF0183
:1065E000EF010280F381E02DDCCF2115310509F1A7
:1065F000281B390B2430310590F412968D919C9113
:1066000013976115710521F0FB019383828304C008
:106610009093A2048093A104FD01329644C0FD0131
:10662000E20FF31F81939193225031092D933C93F4
:106630003AC020919F043091A004232B41F4209173
:106640000801309109013093A00420939F04209108
:106650000601309107012115310541F42DB73EB7F0
:1066600040910A0150910B01241B350BE0919F04CE
:10667000F091A004E217F307A0F42E1B3F0B28179C
:10668000390778F0AC014E5F5F4F2417350748F0AB
:106690004E0F5F1F5093A00440939F0481939193EA
:1066A00002C0E0E0F0E0CF01DF91CF9108950F93B9
:1066B0001F93CF93DF93009709F48CC0FC013297AE
:1066C000138212820091A1041091A20401151105F8
:1066D00081F420813181820F931F20919F0430919A
:1066E000A0042817390779F5F093A004E0939F04DC
:1066F00071C0D80140E050E0AE17BF0750F41296C9
:106700002D913C911397AD012115310509F1D90166
:10671000F3CF9D01DA013383228360817181860F7B
:10672000971F8217930769F4EC0128813981260F9E
:10673000371F2E5F3F4F318320838A819B81938354
:106740008283452B29F4F093A204E093A10442C074
:106750001396FC93EE931297ED01499159919E0186
:10676000240F351FE217F30771F480819181840FA4
:10677000951F029611969C938E9382819381139616
:106780009C938E931297E0E0F0E0D80112968D91E1
:106790009C911397009719F0F8018C01F6CF8D9119
:1067A0009C9198012E5F3F4F820F931F20919F0471
:1067B0003091A0042817390769F4309729F4109212
:1067C000A2041092A10402C0138212821093A004AA
:1067D00000939F04DF91CF911F910F91089581E065
:1067E00090E0F8940C94E5348F929F92AF92BF9210
:1067F000CF92DF92EF92FF92CF93DF93EC0168810B
:1068000079818A819B81611571058105910521F44A
:1068100064E279ED8BE597E02DE133EF41E050E064
:106820000E94823449015A019B01AC01A7EAB1E4FC
:106830000E94A1346B017C01ACEEB4EFA501940180
:106840000E94AF34DC01CB018C0D9D1DAE1DBF1D20
:10685000B7FF03C00197A109B04888839983AA8331
:10686000BB839F77DF91CF91FF90EF90DF90CF9028
:10687000BF90AF909F908F9008950E94F433089539
:106880008CE091E00E94F4330895A0E0B0E08093A2
:106890000C0190930D01A0930E01B0930F01089588
:1068A000DC01CB01FC01F999FECF06C0F2BDE1BDD0
:1068B000F89A319600B40D9241505040B8F70895BF
:1068C000DC01A40FB51F4150504048F0CB01840FAC
:1068D000951F2E910E94713441505040D0F7089579
:1068E000262FF999FECF92BD81BDF89A019700B489
:1068F000021639F01FBA20BD0FB6F894FA9AF99A29
:106900000FBE0895052E97FB1EF400940E94993443
:1069100057FD07D00E94B43407FC03D04EF40C940A
:10692000993450954095309521953F4F4F4F5F4F8B
:10693000089590958095709561957F4F8F4F9F4FEB
:1069400008950E94D634A59F900DB49F900DA49FEA
:10695000800D911D11240895B7FF0C94A1340E945D
:10696000A134821B930B0895A1E21A2EAA1BBB1B14
:10697000FD010DC0AA1FBB1FEE1FFF1FA217B3070B
:10698000E407F50720F0A21BB30BE40BF50B661F21
:10699000771F881F991F1A9469F7609570958095E5
:1069A00090959B01AC01BD01CF010895A29FB0015C
:1069B000B39FC001A39F700D811D1124911DB29F33
:1069C000700D811D1124911D08951DE0CAEFDDE0B9
:1069D00004C0FE010E945E312196CB3FD107C9F76A
:0469E000F894FFCF59
:1069E40070040104FF010000A30480000100000002
:1069F4000503000205010405000102030506000069
:106A040000007010F10FC90F0B31FEFF00001731A9
:106A1400000000003012EC11A00EE2147811250ED3
:106A2400BE2BAB2BA52B0E2C242CFEFF00000B2C15
:086A3400BB2BA82B212C2E2CFA
:00000001FF
